:1000000075817F7401F58F538EF1438E10C2D4C277
:04001000D302003ED9
:0300230002A40232
:03002B0002A43DEF
:0300330002A3D352
:10003B0002A3B1C204753E00753F00D291C2B7C294
:10004B00B6C2B57550FF7551FFD2A1D2B2D2B3C2B1
:10005B00167541FF75427FC217C218C219C21AC268
:10006B001BC21CC21DC21EC21FC220C221C222D271
:10007B0023D224D225D226D227D228D229D22AD2B1
:10008B002BD22CD22DD22EC254C253D253C232C237
:10009B0056C257D233D247C236C237C258C259C2E0
:1000AB005EC25DC238C239C20CC24DD23AD23BC21B
:1000BB003C756C00756D00756F00756E0075717F0A
:1000CB0075707FC24AC24BD24CD24EC24F7567007D
:1000DB00756800C209C20EC20BD20DC20F75690042
:1000EB0075440075450075460075470075480075E9
:1000FB004900754A00754B00754C00754D00754EE7
:10010B0000754F00D212D213755B00755C00755DE4
:10011B0000755E00756100756200756300756400A3
:10012B0075730675740075760675770075431875CB
:10013B007901757A01740090003FF0900040F074E3
:10014B003E900041F07400900072F0900073F090BC
:10015B000074F0900075F0900076F07401900161DE
:10016B00F0900162F0900163F07400900160F090E8
:10017B000164F07401900168F0900166F0900167E2
:10018B00F090016EF0900169F090016AF090016BB4
:10019B00F090016CF090016DF0900170F090016F98
:1001AB00F0900172F01296DB9001C27400F074F0C3
:1001BB00900182F0749F900183F074C3900199F0C9
:1001CB00740390019AF09006DA7400F074179000A3
:1001DB0077F07405900078F0740F900079F074014B
:1001EB00900171F07400900135F0900136F09001A0
:1001FB0037F0900138F0900139F090013AF01297F6
:10020B000C12971512971E1297271297421296BC33
:10021B007400900202F0740090029BF01296C87466
:10022B00009004B7F07400900550F0740C79FF90B7
:10023B00029CF0A3F0D9FC740C79FF90039CF0A303
:10024B00F0D9FC740090049CF0740090049DF07441
:10025B000C79FF900551F0A3F0D9FC740090065176
:10026B00F07400900652F074009006BCF07400908D
:10027B0006C6F09006C7F09006C8F09006C9F0903D
:10028B0006CAF09006CBF09006CCF09006CF740027
:10029B00F012661C1266517550FF7551FF127E26C7
:1002AB007552001290E2128A02753D0012A38A1257
:1002BB00A3A712A3485350DF128BE0128D7D75500C
:1002CB00FF7551FF128B61128E99128EA9122D6E32
:1002DB001237B27402900167F012481E740390013A
:1002EB0067F012481E7404900167F012481E7405E3
:1002FB00900167F012481E7406900167F012481EB9
:10030B007407900167F012481E7408900167F01291
:10031B00481E7401900167F012481E9001E8E0A29C
:10032B00E19250A2E2925A128E5C9001E3E09006A9
:10033B00CDF09001E4E09006CEF01228C6122B2AE5
:10034B00122AD51287EA12A2DE539EE290068A7415
:10035B0000F0C203C20212109B020361783279FFD4
:10036B000000D9FCD8F822784B79FF0000D9FCD8D3
:10037B00F82278327932D9FED8FA22F87902D9F6F6
:10038B00D8F222E627F52C0809E637F52D782C2232
:10039B00C3E697F52C0809E697F52D782C22862CC9
:0E03AB00872E0809862D872F12042E78312206
:1003B9008631088632088633088634872E09872FC6
:1003C9001203D1782C793322753500753610120451
:1003D900131203E4120407D536F422C3E533952E2C
:1003E900E534952FE5359400500122E533952EF536
:1003F90033E534952FF534E5359400F53522B3E529
:100409002C33F52CE52D33F52D22C3E53133F531A8
:10041900E53233F532E53333F533E53433F534E595
:100429003533F53522E52C852EF0A4F53185F032EA
:10043900E52D852FF0A4F53385F034E52D852EF0D3
:10044900A42532F532E53335F0F533E5343400F5DA
:1004590034E52C852FF0A42532F532E53335F0F556
:1004690033E5343400F53422E582C4540FF9E583C9
:10047900C46922E5820303543FF9E583030354C0A9
:1004890069227A0CC297D2A3A29633C933C9C2A3EF
:10049900DAF2F8D29722C2A3C2973392A6D2A3DA8C
:1004A900F5C2A312048BE95403F9227A0574E01208
:1004B900049FF5838882227A0574D812049FF583F4
:1004C9008882227A0574C012049FF5838882227A71
:1004D9000574C812049FF5838882227A0574D012A4
:1004E900049FF5838882227A0574E812049FF583B4
:1004F9008882227A0574F012049FF5838882227A11
:100509000574F812049FF583888222C2B412052467
:100519001205711205BED2B4C2B422A846A947E990
:10052900540F44507A08C2A1C2A33392A6D2A3DAC7
:10053900F77A08E8C2A33392A6D2A3DAF7C2A3D204
:10054900A1A844A945E9540F44D07A08C2A1C2A37D
:100559003392A6D2A3DAF77A08E8C2A33392A6D2D5
:10056900A3DAF7C2A3D2A122A84AA94BE9540F449E
:10057900507A08C2B2C2A33392A6D2A3DAF77A0894
:10058900E8C2A33392A6D2A3DAF7C2A3D2B2A84E85
:10059900A94FE9540F44D07A08C2B2C2A33392A634
:1005A900D2A3DAF77A08E8C2A33392A6D2A3DAF77C
:1005B900C2A3D2B222A848A949E9540F44507A08E3
:1005C900C2B3C2A33392A6D2A3DAF77A08E8C2A3C8
:1005D9003392A6D2A3DAF7C2A3D2B3A84CA94DE9A4
:1005E900540F44D07A08C2B3C2A33392A6D2A3DA75
:1005F900F77A08E8C2A33392A6D2A3DAF7C2A3D244
:10060900B322F5377538007837753B22753C007988
:100619003B1203A9868208868322F537753800784C
:1006290037753B44753C00793B1203A986820886DD
:100639008322F5377538007837753B20753C00798A
:100649003B1203A986820886832220A204753E00F4
:100659002220A003D20422753E0122E53EB53F04C3
:10066900853E3F22B4001520040A0540853E3FD24D
:1006790006D20222C204853E3FD2062220040A1570
:1006890040853E3FD206D20322C204853E3FD206B0
:1006990022E56B20E601229006CFE070030206BE38
:1006A900020707E56B20E601229006CFE0700302FE
:1006B90007500207999006D0E01475F006A4900639
:1006C900CB739001820207E29001820207E2900156
:1006D900820208089001820208189001820207E24A
:1006E9009001820207E29001820207E290018202F0
:1006F90007E29001820207E29001820207E2900676
:10070900D0E01475F006A4900714739001830207D2
:10071900E29001830207FB90018302086C90018338
:0E07290002086C90018302082E9001830208E2
:1007370032900183020839900183020808900183EF
:100747000208439001830208569006D1E01475F021
:1007570006A490075D739001990207E29001990240
:1007670007E2900199020808900199020818900180
:10077700990207E29001990207E29001990207E2C4
:100787009001990207E29001990207E2900199020C
:1007970007E29006D1E01475F006A49007A67390BF
:1007A700019A0207E290019A0207FB90019A020858
:1007B7006C90019A02086C90019A02082E90019A97
:1007C70002083290019A02083990019A02080890AB
:1007D700019A02084390019A02085612086D1208FE
:1007E7008612089F1208B81208D11208EA120903E4
:1007F70012091C2212086D12088612089F1208B8E7
:100807002212086D12088612089F1208B81208D122
:100817002212086D12088612089F1208B81208D112
:100827001208EA1209032212086D2212086D120833
:10083700862212086D12088612089F2212086D126E
:10084700088612089F1208B81208D11208EA221265
:10085700086D12088612089F1208B81208D11208EC
:10086700EA1209032222E56B30E108C21720230EA2
:10087700D22322C223201706D217E0B2E7F022E5DF
:100887006B30E208C21820240ED22422C22420187A
:1008970006D218E0B2E6F022E56B30E308C2192071
:1008A700250ED22522C225201906D219E0B2E5F07D
:1008B70022E56A30E108C21A20260ED22622C22675
:1008C700201A06D21AE0B2E4F022E56A30E208C242
:1008D7001B20270ED22722C227201B06D21BE0B2DD
:1008E700E3F022E56A30E308C21C20280ED2282252
:1008F700C228201C06D21CE0B2E2F022E56A30E5ED
:1009070008C21D20290ED22922C229201D06D21D68
:10091700E0B2E1F022E56A30E708C21E202A0ED2D3
:100927002A22C22A201E06D21EE0B2E0F022E56A81
:1009370030E40630E611C2382230380122D238902E
:1009470006CFE07400F02230380122D2389006CF6B
:10095700E07401F0229006CFE07009E551C2E3D2BE
:10096700E5F55122E551D2E3C2E5F55122120A3BE2
:100977009006CFE070079001821209A222900183AE
:100987001209A222120A3B9006CFE0700790019944
:100997001209A22290019A1209A222E020E709E592
:1009A70050D2E1F5500209B5E550C2E1F550E0201B
:1009B700E609E550D2E2F5500209C8E550C2E2F572
:1009C70050E020E509E550D2E3F5500209DBE55098
:1009D700C2E3F550E020E409E550D2E6F5500209FC
:1009E700EEE550C2E6F550E020E309E550D2E7F521
:1009F70050020A01E550C2E7F550E020E209E5514F
:100A0700D2E1F551020A14E551C2E1F551E020E1C6
:100A170009E551D2E4F551020A27E551C2E4F5513F
:100A2700E020E009E551D2E7F551020A3AE551C263
:100A3700E7F55122E550D2E4F550E551D2E0D2E294
:100A4700D2E6F55122B4FF03740022B4EB01225021
:100A5700012274EB22B40101225003740122B4EC89
:100A6700012250012274EC22B4FF03740022B40C5B
:100A77000122500122740C22B40101225003740197
:100A870022B4100122500122741022B40101225015
:100A970003740122B40A0122500122740A22B4010C
:0E0AA70001225003740122B4200122500122CA
:100AB500742022B40101225003740122B41F0122C3
:100AC500500122741F22B40101225003740122B483
:100AD500080122500122740822B401012250037436
:100AE5000122B4110122500122741122B401012204
:100AF5005003740122B47F0122500122747F22B475
:100B0500FF03740022B4030122500122740322B4AE
:100B1500EB012250012274EB22B40101225003742F
:100B25000122B40A0122500122740A22B4010122D1
:100B35005003740122B40C0122500122740C22B41A
:100B45000101225003740122B403012250012274D1
:100B55000322B40101225003740122B4040122507E
:100B65000122740422B40101225003740122B4034A
:100B75000122500122740322B401012250037401A1
:100B850022B4050122500122740522B4010122502C
:100B950003740122B4030122500122740322B4011B
:100BA50001225003740122B403012250012274036F
:100BB50022B40101225003740122B406012250011E
:100BC50022740622B40101225003740122B41901D2
:100BD50022500122741922B401012250037401220A
:100BE500B4220122500122742222B40101225003B1
:100BF500740122B40A0122500122740A22B40101AF
:100C0500225003740122B4070122500122740722E5
:100C1500B4FF03740022B47E0122500122747E22A7
:100C2500B40301225003740322B48F012250012220
:100C3500748F22B40101225003740122B4030122EE
:100C4500500122740322B40101225003740122B41D
:100C5500020122500122740222B4010122500374C0
:100C65000122B4020122500122740222B4010122A0
:100C75005003740122B4020122500122740222B4ED
:100C85000101225003740122B40301225001227490
:100C95000322B40101225003740122B45F012250E2
:100CA5000122745F22B4FF08B9000374FE227400A8
:100CB50022B40101225003740122B4110122500112
:100CC50022741122B40101225003740122B40501DA
:100CD50022500122740522B401012250037401221D
:100CE500B40B0122500122740B22B40101225003DE
:100CF500740122B57C0122500122E57C22B4010158
:100D0500225003740122B43A0122500122743A227E
:100D1500B40101225003740122B44601225001227C
:100D2500744622B40101225003740122B4800122C9
:100D3500500122748022B40101225003740122B4AF
:100D4500070122500122740722B4010122500374C5
:100D55000122B40C0122500122740C22B40101229B
:100D65005003740122B40C0122500122740C22B4E8
:100D75000101225003740122B40C01225001227496
:100D85000C22B40101225003740122B41701225030
:100D95000122741722300909C209300A02C20AD297
:100DA5000B22305F09C25F300A02C20AD20B223021
:100DB5005015E56B30E61030E003C20C22200C071D
:100DC500D20CB20E120DCD22300E0AD20AD20ED29C
:100DD5000F5350DF22D20DC20EC20B43502022907A
:100DE5000173E02414FA74003400FB7537D07538AC
:100DF50012753913753A0078378A3B8B3C793B126B
:100E050003B9E6F54108E6F54222D211F59920111C
:100E1500FD22B4F808300A02C20AD20B22B4FA0A3B
:0E0E2500D20AD20ED20F5350DF22B4FC0AD2F2
:100E33000DC20EC20B43502022B4FB09D20AD20EBC
:100E4300D20F5350DF22B4F0077567007568002294
:100E5300B4F10775670075680022B4F2077567007F
:100E630075680022B4F30F7567007568002230506F
:100E73000122120E172250F6E5692490F57EE9B59A
:100E83007E08756701C251C25522E5692480F57E4B
:100E9300E9B57E08756801D251C25522E56924B0CF
:100EA300F57EE9B57E06756701D2552230E70D75EB
:100EB300670075680022020EFE020F142055FA2007
:100EC30051F4A967B9000122A967B901050567F5BE
:100ED3006522B9021405676008E565120F42D24F17
:100EE30022E565121040D24F22B903050567F56567
:100EF30022B90406756701020EDA22A968B9000156
:100F030022A968B901070568F565020EE475680151
:100F130022A967B9000122A967B901050567F57F11
:100F230022B902090567F9120F46D24F22B9030508
:100F33000567F57F22B90406756701020F2922129E
:100F4300100D22E57FB41403020F58500122B41E82
:100F53000122400122C3941475F003A4900F63731C
:100F6300020F81020F8A020F98020FA8020FB70225
:100F73000FC7020FD0020FDE020FEE020FFDE912C0
:100F83000C15900177F022E975F00C8404120CDC47
:100F930090017AF022E975F00E8404120BEF9001B0
:100FA30075F0D23222E975F00584120BC9900174F1
:100FB300F0D23222E975F00F8404120CC990017645
:100FC300F0D23222E9120C1590018EF022E975F06D
:100FD3000C8404120CDC900191F022E975F00E846C
:100FE30004120BEF90018CF0D23222E975F00584E4
:100FF300120BC990018BF0D23222E975F00F8404F1
:10100300120CC990018DF0D23222B42414C394245B
:10101300FF90020F121077E0D2E7F01287F5D23279
:101023002250EAB40B012240FDC3940CFF9004C488
:10103300121095E0D2E7F01288A7D23222303A019B
:1010430022B42414C39424FF90020F121077E0C239
:10105300E7F012880DD2322250EAB40B012240FD90
:10106300C3940CFF9004C4121095E0C2E7F01288F9
:10107300BFD23222128659EF240C858237858338FA
:101083007837F53B753C00793B12038E86820886E0
:10109300832212866702107A129A1E129A51129EA6
:1010A3006212A25A12A2C11233E91286C712874BE7
:1010B300127E821290FE129522124AB01284F71207
:1010C300661C12270D120DB43050139001E7E0B4E3
:1010D3000306120DA70210E1120DE4120D9A126617
:1010E3001C200D03021103C20D9001E6E0B40103BD
:1010F3000210FB74FC120E0F1211EDC2B71293E132
:10110300300F46C20F9001E6E0B4010302111774D9
:10111300FA120E0F1211EDC24C12852012571890BD
:10112300049DE01490049CF0125ED6900652E014E5
:10113300900651F0E550C2E5F550D2B7121DB41236
:10114300939912119AC24AC24B300A0302109B2090
:101153000E03021199200B03021199C20B9001E6B1
:10116300E0B4010302117FB4020874F8120E0F02F7
:10117300117FB25C305C0574F8120E0F20500B30F7
:101183005A08B25B305B03021199121DC712209FEC
:1011930012123E12119A22121DF3121EFD129356C1
:0E11A3001220CB1221D51223777E0112240CCC
:1011B1001224BC7E0212240C1224BC7E0312240CC5
:1011C1001224BC7E0412240C1224BC7E0512240CB1
:1011D1001224BC7E0612240C1224BC7E0712240C9D
:1011E1001224BC7E0812240C1224BC22435020126B
:1011F1001F1B1221F37400900077F0900135F090DD
:101201000137F0900138F090013AF07552001297D1
:101211000C12971512971E1297271298AD900188FC
:10122100E014A3F01298F890019FE014A3F0C256C5
:10123100C25790015F7400F0C25BC25C2212166754
:1012410012167C1216961216C41216DE1216F81217
:10125100171212172C12174C121766121780121739
:101261009A1217B41217CE1217E812180212181C8C
:1012710022B4010490007A22B4020490007C22B4CA
:10128100030490007E22B4040490008022B406047A
:1012910090008222B4080490008422B409049000D2
:1012A1008622B40C0490008822B4100490008A2293
:1012B100B4120490008C22B4180490008E22B42041
:1012C1000490009022B4240490009222B43004903F
:1012D100009422B4400490009622B44804900098EF
:1012E1002290009A22E01475F004A49012F073EF9A
:1012F100021365EF021533EF0213B2EF0213FFEF92
:1013010002144CEF021499EF0214E6EF021580EF7C
:101311000215CDEF02161A1475F004A4901321736F
:1013210090007A2290007E229000822290008822F2
:1013310090008E229000942290009A2290007C22AC
:10134100900080229000842290008A2290009022B6
:10135100900096229000862290008C22900092228A
:10136100900098221475F004A490136E7390007B82
:101371002290007F22900083229000892290008F8A
:10138100229000952290009B2290007D2290008166
:10139100229000852290008B22900091229000974C
:1013A100229000872290008D229000932290009934
:1013B100221475F004A49013BB7390009C2290003A
:1013C1009E229000A0229000A3229000A6229000CD
:1013D100A9229000AC2290009D2290009F229000B3
:1013E100A1229000A4229000A7229000AA2290009E
:1013F100A2229000A5229000A8229000AB22147591
:10140100F004A4901408739000AD229000AF2290D4
:1014110000B1229000B4229000B7229000BA22902D
:1014210000BD229000AE229000B0229000B2229026
:1014310000B5229000B8229000BB229000B3229008
:1014410000B6229000B9229000BC221475F004A4C9
:10145100901455739000BE229000C0229000C222C9
:101461009000C5229000C8229000CB229000CE228D
:101471009000BF229000C1229000C3229000C6229A
:101481009000C9229000CC229000C4229000C72273
:101491009000CA229000CD221475F004A49014A2E9
:1014A100739000CF229000D1229000D3229000D6D9
:1014B100229000D9229000DC229000DF229000D0FF
:1014C100229000D2229000D4229000D7229000DAFC
:1014D100229000DD229000D5229000D8229000DBDE
:1014E100229000DE221475F004A49014EF73900092
:1014F100E0229000E2229000E4229000E722900096
:10150100EA229000ED229000F0229000E12290006A
:10151100E3229000E5229000E8229000EB22900067
:0E152100EE229000E6229000E9229000EC22DB
:10152F009000EF221475F004A490153C739000F115
:10153F00229000F3229000F5229000F8229000FBF9
:10154F00229000FE22900101229000F2229000F4DE
:10155F00229000F6229000F9229000FC229000FFCA
:10156F00229000F7229000FA229000FD22900100B5
:10157F00221475F004A49015897390010222900132
:10158F000422900106229001092290010C22900161
:10159F000F22900112229001032290010522900147
:1015AF00072290010A2290010D2290011022900132
:1015BF00082290010B2290010E2290011122147526
:1015CF00F004A49015D67390011322900115229068
:1015DF0001172290011A2290011D229001202290C2
:1015EF0001232290011422900116229001182290BB
:1015FF00011B2290011E229001212290011922909D
:10160F00011C2290011F22900122221475F004A4C4
:10161F0090162373900124229001262290012822F4
:10162F0090012B2290012E22900131229001342221
:10163F0090012522900127229001292290012C222E
:10164F0090012F229001322290012A2290012D2207
:10165F00900130229001332290007A7400F012181A
:10166F003990007BE004B410027400F02290007CEB
:10167F00E004B402107400F012188B90007DE004A7
:10168F00B410027400F02290007EE004B4032474BE
:10169F0000F0B2B790017EE0B40202C2B69001959D
:1016AF00E0B40202C2B51218DD90007FE004B4105E
:1016BF00027400F022900080E004B404107400F073
:1016CF0012192F900081E004B410027400F02290E0
:1016DF000082E004B406107400F0121981900083A8
:1016EF00E004B410027400F022900084E004B40807
:1016FF00107400F01219D3900085E004B410027436
:10170F0000F022900086E004B409107400F0121A61
:10171F0025900087E004B410027400F02290008836
:10172F00E004B40C167400F0E550B2E5F550121A4F
:10173F0077900089E004B410027400F02290008AC0
:10174F00E004B410107400F0121AC990008BE0047A
:10175F00B410027400F02290008CE004B4121074E4
:10176F0000F0121B1B90008DE004B410027400F007
:10177F002290008EE004B418107400F0121B6D90CC
:10178F00008FE004B410027400F022900090E00487
:10179F00B420107400F0121BBF900091E004B4103D
:1017AF00027400F022900092E004B424107400F050
:1017BF00121C11900093E004B410027400F02290F8
:1017CF000094E004B430107400F0121C6390009584
:1017DF00E004B410027400F022900096E004B440CC
:1017EF00107400F0121CB5900097E004B41002744E
:1017FF0000F022900098E004B448107400F0121D1D
:10180F0007900099E004B410027400F02290009A3F
:10181F00E004B460137400F0121DB4121D5990004F
:10182F009BE004B410027400F02290009C757C05BC
:10183F00121DAB9000AD757C07121DAB9000BE75ED
:10184F007C09121DAB9000CF757C0A121DAB900066
:10185F00E0757C0B121DAB9000F1757C0C121DAB6B
:10186F00900102757C0D121DAB900113757C0E1249
:10187F001DAB900124757C0F121DAB2290009D753E
:10188F007C05121DAB9000AE757C07121DAB90004E
:0E189F00BF757C09121DAB9000D0757C0A123B
:1018AD001DAB9000E1757C0B121DAB9000F2757CA9
:1018BD000C121DAB900103757C0D121DAB90011424
:1018CD00757C0E121DAB900125757C0F121DAB2280
:1018DD0090009E757C05121DAB9000AF757C0712B4
:1018ED001DAB9000C0757C09121DAB9000D1757CAD
:1018FD000A121DAB9000E2757C0B121DAB9000F32C
:10190D00757C0C121DAB900104757C0D121DAB90F6
:10191D000115757C0E121DAB900126757C0F121DE5
:10192D00AB2290009F757C05121DAB9000B0757CAD
:10193D0007121DAB9000C1757C09121DAB9000D232
:10194D00757C0A121DAB9000E3757C0B121DAB90DC
:10195D0000F4757C0C121DAB900105757C0D121DEC
:10196D00AB900116757C0E121DAB900127757C0F87
:10197D00121DAB229000A0757C05121DAB9000B11D
:10198D00757C07121DAB9000C2757C09121DAB90C2
:10199D0000D3757C0A121DAB9000E4757C0B121DF3
:1019AD00AB9000F5757C0C121DAB900106757C0D8E
:1019BD00121DAB900117757C0E121DAB9001287591
:1019CD007C0F121DAB229000A1757C05121DAB90F2
:1019DD0000B2757C07121DAB9000C3757C09121DFA
:1019ED00AB9000D4757C0A121DAB9000E5757C0B95
:1019FD00121DAB9000F6757C0C121DAB9001077596
:101A0D007C0D121DAB900118757C0E121DAB900153
:101A1D0029757C0F121DAB229000A2757C05121D3D
:101A2D00AB9000B3757C07121DAB9000C4757C099B
:101A3D00121DAB9000D5757C0A121DAB9000E6759A
:101A4D007C0B121DAB9000F7757C0C121DAB900139
:101A5D0008757C0D121DAB900119757C0E121DAB16
:101A6D0090012A757C0F121DAB229000A3757C0589
:101A7D00121DAB9000B4757C07121DAB9000C5759F
:101A8D007C09121DAB9000D6757C0A121DAB90001F
:101A9D00E7757C0B121DAB9000F8757C0C121DAB1D
:101AAD00900109757C0D121DAB90011A757C0E12FB
:101ABD001DAB90012B757C0F121DAB229000A475F0
:101ACD007C05121DAB9000B5757C07121DAB900007
:101ADD00C6757C09121DAB9000D7757C0A121DAB23
:101AED009000E8757C0B121DAB9000F9757C0C1203
:101AFD001DAB90010A757C0D121DAB90011B757C01
:101B0D000E121DAB90012C757C0F121DAB22900097
:101B1D00A5757C05121DAB9000B6757C07121DAB2B
:101B2D009000C7757C09121DAB9000D8757C0A1208
:101B3D001DAB9000E9757C0B121DAB9000FA757C06
:101B4D000C121DAB90010B757C0D121DAB90011C81
:101B5D00757C0E121DAB90012D757C0F121DAB22E5
:101B6D009000A6757C05121DAB9000B7757C071211
:101B7D001DAB9000C8757C09121DAB9000D9757C0A
:101B8D000A121DAB9000EA757C0B121DAB9000FB89
:101B9D00757C0C121DAB90010C757C0D121DAB905C
:101BAD00011D757C0E121DAB90012E757C0F121D43
:101BBD00AB229000A7757C05121DAB9000B8757C0B
:101BCD0007121DAB9000C9757C09121DAB9000DA90
:101BDD00757C0A121DAB9000EB757C0B121DAB9042
:101BED0000FC757C0C121DAB90010D757C0D121D4A
:101BFD00AB90011E757C0E121DAB90012F757C0FE5
:101C0D00121DAB229000A8757C05121DAB9000B97A
:0E1C1D00757C07121DAB9000CA757C09121D64
:101C2B00AB9000DB757C0A121DAB9000EC757C0B46
:101C3B00121DAB9000FD757C0C121DAB90010E7547
:101C4B007C0D121DAB90011F757C0E121DAB90010C
:101C5B0030757C0F121DAB229000A9757C05121DEF
:101C6B00AB9000BA757C07121DAB9000CB757C094D
:101C7B00121DAB9000DC757C0A121DAB9000ED754C
:101C8B007C0B121DAB9000FE757C0C121DAB9001F2
:101C9B000F757C0D121DAB900120757C0E121DABC8
:101CAB00900131757C0F121DAB229000AA757C053B
:101CBB00121DAB9000BB757C07121DAB9000CC7551
:101CCB007C09121DAB9000DD757C0A121DAB9000D8
:101CDB00EE757C0B121DAB9000FF757C0C121DABCF
:101CEB00900110757C0D121DAB900121757C0E12AD
:101CFB001DAB900132757C0F121DAB229000AB75A2
:101D0B007C05121DAB9000BC757C07121DAB9000BF
:101D1B00CD757C09121DAB9000DE757C0A121DABD4
:101D2B009000EF757C0B121DAB900100757C0C12B3
:101D3B001DAB900111757C0D121DAB900122757CB2
:101D4B000E121DAB900133757C0F121DAB22900050
:101D5B00AC757C05121DAB9000BD757C07121DABDD
:101D6B009000CE757C09121DAB9000DF757C0A12BA
:101D7B001DAB9000F0757C0B121DAB900101757CB7
:101D8B000C121DAB900112757C0D121DAB90012333
:101D9B00757C0E121DAB900134757C0F121DAB229E
:101DAB00E004B57C027400F02290017EE0B40202E4
:101DBB00D2B6900195E0B40202D2B522304A0BC2E2
:101DCB004A90049DE01490049CF022900179E0125B
:101DDB001318E0900135F0900179E0FF9006D012D6
:101DEB0012E6E0900137F022121DD6900135E0B4D7
:101DFB000003121E0122900137E07012F990017D51
:101E0B00E0B4030990049DE01490049CF0E90412E3
:101E1B001E6A227400900137F0C2482274009001B0
:101E2B0035F022740090049CF022B40803021E3D8E
:101E3B005012F9900178E075F002A414149072A07E
:101E4B0093021E61C39408F9900178E075F002A427
:101E5B0014149072A19323D9FDA2E0121E8B22B40D
:101E6B000803021E725008F9900182E0021E82C321
:101E7B009408F9900183E023D9FDA2E0121E8B2276
:101E8B00400E90017CE014700122D2481256992228
:101E9B00D2481231BC7400900136F012569990065C
:101EAB00BCE02BF573900177E06006121ECC021E8E
:101EBB00C2122047121EE990017EE0B40102D2B695
:101ECB0022122047E573B57403021EE95005C214B4
:101EDB00021EE0D214121F28C21285737422D21272
:101EEB00E573F57412060BC2AD858244858345D22A
:101EFB00AD22900136E0F57C900187E0B57C0412B1
:101F0B001F1B2240FA121F1422900136E004F0220C
:101F1B0012208590017EE0B40102C2B62220142C5F
:101F2B00E57412060BC2AD858244858345D2ADE5BF
:101F3B0074C39573F57912060B858259E58270038C
:101F4B0075590185835A055A121F8322E5741206AF
:101F5B000BC2AD858244858345D2ADE573C39574C1
:101F6B00F57912060B858259E58270037559018547
:101F7B00835A055A121F8322900177E0FA7480C3AB
:101F8B009AF5437537F175384E753904753A007803
:0E1F9B003785793B753C00793B1203B98637D8
:101FA900088638753900753A00783785433B753CA2
:101FB90000793B1203B98637088638753900753AB6
:101FC900007837900173E02414F53B753C00793BA8
:101FD9001203B98682088683C2AD85825BE5827069
:101FE90003755B0185835C055C855B5D855C5ED201
:101FF900AD22D55905D55A03D212227559FF22307F
:1020090012012220140302202C121FFB301201227C
:10201900E5442401F582E5453400F583858244854C
:10202900834522121FFB30120122C3E5449401F5B6
:1020390082E5459400F58385824485834522900293
:102049009BE07004122085221298ADF57090017FF3
:10205900E0B4010FE57012063BC2AD85824C858361
:102069004DD2AD1220857490120E0FE5732424C24F
:10207900E7120E0FE570120E0FD23422203401221E
:102089007490120E0FE5742424C2E7120E0F740027
:10209900120E0FC23422304B0BC24B900652E01481
:1020A900900651F022900190E0121318E090013847
:1020B900F0900190E0FF9006D11212E6E090013A0B
:1020C900F0221220AE900138E0B400031220D92288
:1020D90090013AE07012F9900194E0B40309900676
:1020E90052E014900651F0E9041221422274009042
:1020F900013AF0C249227400900138F0227400902C
:102109000651F022B408030221155012F990018FEB
:10211900E075F002A414149072A093022139C394BB
:1021290008F990018FE075F002A414149072A1933C
:1021390023D9FDA2E012216322B4080302214A50E7
:1021490008F9900199E002215AC39408F990019A7B
:10215900E023D9FDA2E012216322400E900193E011
:1021690014700122D249125E5722D249123A0974D7
:1021790000900139F0125E579006BCE02BF576907D
:10218900018EE060061221A402219A12231F122156
:10219900C1900195E0B40102D2B52212231FE57660
:1021A900B57703021EE95005C2150221B8D21512EE
:1021B9002200C21385767722D213E576F5771206C7
:1021C9000BC2AD858246858347D2AD22900139E0A5
:1021D900F57C90019EE0B57C041221F32240FA12AD
:1021E90021EC22900139E004F02212235D9001953F
:1021F900E0B40102C2B52220152CE57712060BC204
:10220900AD858246858347D2ADE577C39576F57A64
:1022190012060B85825FE5827003755F0185836015
:10222900056012225B22E57712060BC2AD85824654
:10223900858347D2ADE576C39577F57A12060B8586
:10224900825FE5827003755F0185836005601222F4
:102259005B2290018EE0FA7480C39AF5437537F1D9
:1022690075384E753904753A007837857A3B753C6F
:1022790000793B1203B98637088638753900753AF3
:1022890000783785433B753C00793B1203B98637A3
:10229900088638753900753A007837900173E0245B
:1022A90014F53B753C00793B1203B9868208868395
:1022B900C2AD858261E5827003756101858362051E
:1022C90062856163856264D2AD22D55F05D56003FD
:0222D900D2131E
:1022DB0022755FFF22301301222015030223041203
:1022EB0022D330130122E5462401F582E547340061
:1022FB00F583858246858347221222D33013012230
:10230B00C3E5469401F582E5479400F58385824643
:10231B0085834722900550E0700412235D221298AA
:10232B00F8F571900196E0B4010FE57112063BC20E
:10233B00AD85824E85834FD2AD12235D7491120E03
:10234B000FE5762424C2E7120E0FE571120E0FD2A1
:10235B003522203501227491120E0FE5772424C209
:10236B00E7120E0F7400120E0FC235227E011223DC
:10237B00A07E021223A07E031223A07E041223A0B0
:10238B007E051223A07E061223A07E071223A07EB9
:10239B00081223A0229001AA1223CCE0121318E0FA
:1023AB0090013B1223CCF09001AA1223CCE0FF90BA
:1023BB0006D21223CC1212E6E090014B1223CCF082
:1023CB0022C0E08582378583387837EE14F53B756C
:1023DB003C00793B12038E8682088683D0E022C0B4
:1023EB00E08582378583387837EE1475F002A4F5D3
:1023FB003B753C00793B12038E8682088683D0E0C6
:10240B002290013B1223CCE0B4000312241A229039
:10241B00014B1223CCE00412247522740090014B63
:10242B001223CCF022740090013B1223CCF022B487
:10243B0008030224425015FF9001A21223CCE07531
:10244B00F002A414149072A09302246CC39408FF9E
:10245B009001A21223CCE075F002A414149072A187
:10246B009323DFFDA2E012249C22B4080302247DF7
:10247B00500BFF9001D31223EAE0022493C394087C
:10248B00FF9001D41223EAE023DFFDA2E012249C8B
:10249B00224001221224B5124A661224B574009010
:1024AB0001431223CCF01224E322900167E0CEF01B
:1024BB00229001431223CCE0F57C9001CB1223CC6C
:1024CB00E0B57C041225302240FA1224D922900167
:1024DB00431223CCE004F022BE0107435201122524
:1024EB007D22BE020743520212259422BE030743EC
:1024FB0052201225AB22BE04074352041225C222DE
:10250B00BE05074352401225D922BE060743520887
:10251B001225F022BE070743528012260722435290
:10252B001012261E22BE01075352FE12263522BE62
:10253B0002075352FD12265022BE03075352DF12DD
:10254B00266B22BE04075352FB12268622BE0507BA
:10255B005352BF1226A122BE06075352F71226BCB6
:10256B0022BE070753527F1226D7225352EF122651
:10257B00F2227499120E0F7424120E0F7464120E41
:10258B000F9006DAE0D2E0F0227499120E0F742548
:10259B00120E0F746E120E0F9006DAE0D2E1F022DB
:1025AB007499120E0F743C120E0F7478120E0F905A
:1025BB0006DAE0D2E2F0227499120E0F743F120E7B
:1025CB000F747F120E0F9006DAE0D2E3F0227499AB
:1025DB00120E0F7430120E0F746E120E0F9006DA6D
:1025EB00E0D2E4F0227499120E0F743B120E0F74AA
:1025FB007F120E0F9006DAE0D2E5F0227499120EDC
:10260B000F743D120E0F747F120E0F9006DAE0D28C
:10261B00E6F0227499120E0F743E120E0F747F1295
:10262B000E0F9006DAE0D2E7F0229006DAE020E017
:10263B000122C2E0F07499120E0F7424120E0F7463
:0E264B0000120E0F229006DAE020E10122C2FA
:10265900E1F07499120E0F7425120E0F7400120E08
:102669000F229006DAE020E20122C2E2F074991208
:102679000E0F743C120E0F7400120E0F229006DA20
:10268900E020E30122C2E3F07499120E0F743F12A5
:102699000E0F7400120E0F229006DAE020E40122D8
:1026A900C2E4F07499120E0F7430120E0F740012F6
:1026B9000E0F229006DAE020E50122C2E5F07499B6
:1026C900120E0F743B120E0F7400120E0F22900699
:1026D900DAE020E60122C2E6F07499120E0F743D89
:1026E900120E0F7400120E0F229006DAE020E70195
:1026F90022C2E7F07499120E0F743E120E0F740085
:10270900120E0F221229CCE56B30E7071227F512BA
:1027190029A1221227D11227E31227262290016626
:10272900E01475F006A49027337390680202276FAE
:1027390090680802276F90680E02276F906814024C
:10274900276F90681A02276F90682002276F906898
:102759002602279490682C02276F90683202276F0F
:102769009068380227B905A29000427B06128B397E
:102779009067CF05A29000487B0A128B399067CFEA
:1027890005A29000527B10128B392205A2900042BB
:102799007B05128B399067CF05A29000477B0B12FE
:1027A9008B399067CF05A29000527B10128B39228A
:1027B90005A29000427B10128B399067CF05A29039
:1027C90000527B10128B392220020122C20590018E
:1027D90066E004120B1EF0C2022220030122C20588
:1027E900900166E014120B1EF0C20322E56B20E58E
:1027F9000122E56B30E60122E56A30E02130E1276C
:1028090030E22730E32730E52730E727E56B30E072
:102819002530E10D30E20430E30A22022842022881
:102829005102286002286F02287E02288D02289C06
:102839000228A50228B40228BD9001727401F0741F
:1028490001900166F00228CA9001727401F07402C5
:10285900900166F00228CA9001727402F074039024
:102869000166F00228CA9001727403F074049001A1
:1028790066F00228CA9001727401F074059001662D
:10288900F00228CA9001727401F07406900166F092
:102899000228CA7407900166F00228CA900172746E
:1028A90001F07408900166F00228CA740990016663
:1028B900F00228CA740A900166F00228CA900166DB
:1028C900E0B40106906802022913B4020690680870
:1028D900022913B40303022921B40403022935B4DC
:1028E900050690681A022913B40606906820022981
:1028F90013B40703022949B4080690682C02295D1C
:10290900B409069068320229132212297105A2908E
:1029190000427B06128B392290680E12297105A29A
:102929009000427B06128B3912297E22906814127C
:10293900297105A29000427B06128B3912297E2249
:1029490090682612297105A29000427B05128B39E5
:102959001246BD2290682C12297105A29000427B73
:1029690005128B39124C152222200801222005015B
:10297900229067EF223053069069D002299620549D
:10298900069069C80229969069CC02299605A290F9
:1029990000477B04128B3922900166E01475F0031D
:1029A900A49029AE73022A08023602023B42023D74
:1029B9003C023FBC0241D90246F2024C4A024EACEB
:0E29C9000252ABE56B30E703C2072220070481
:1029D700B208D2072220020122C205900168E00452
:1029E700120B31F0900169F0C2022220030122C2CA
:1029F70005900168E014120B31F0900169F0C203F1
:102A070022E56B20E50122C2541287EA122B2A1213
:102A17002AD53008071229DC1229F222900168E032
:102A2700B4010A122BA7122BBB12855722B4020A34
:102A370012300812301C12855722B4030A1230AA2A
:102A47001230BE12855722B4040A1230F712310928
:102A570012855722B4051F122C8F122CA812069A22
:102A670012097412093512095C9001727404F0900E
:102A770001637401F022B4060A122EED122F01121F
:102A8700855722B4070A12314D12315F128557223A
:102A9700B4080A1231FA12320C12855722B4090A05
:102AA7001232BC1232CE12855722B40A0A123304EC
:102AB70012331612855722B40B0A12335212336699
:102AC700128557221233A41233B61285572290016A
:102AD70068E0B40104122BCF22B402041230302272
:102AE700B403041230D222B4040412311B22B405F9
:102AF70004122D4A22B40604122F2D22B407041201
:102B0700317122B4080412321E22B409041232E0D1
:102B170022B40A0412332822B40B0412337A221285
:102B270033C822900168E01475F006A4902B377320
:102B3700906A46022B7F906A50022B7F906A5A0256
:102B47002B7F906A64022B7F906A6E022B8D906AAE
:102B570078022B7F906A82022B7F906A8C022B7FF0
:102B6700906A96022B7F906AA0022B7F906AAA0236
:102B77002B7F906AB4022B7F122B9B05A2900048F3
:102B87007B0A128B3922122B9B05A29000487B05EA
:102B9700128B392220080122200501229067EF229B
:102BA70020020122C205900174E004120BC9F0C291
:102BB70002D2322220030122C205900174E01412CE
:102BC7000BC9F0C203D23222900174E01475F006EB
:102BD700A4902BDC73906C3E022C84906C4E022CDC
:102BE70084906C5E022C84906C6E022C84906C7EB8
:102BF700022C84906C8E022C84906C9E022C849004
:102C07006CAE022C84906CBE022C84906CCE022C8D
:102C170084906CDE022C84906CEE022C84906CFE07
:102C2700022C84906D0E022C84906D1E022C8490D1
:102C37006D2E022C84906D3E022C84906D4E022CDA
:102C470084906D5E022C84906D6E022C84906D7E54
:102C5700022C84906D8E022C84906D9E022C8490A1
:102C67006DAE022C84906DBE022C84906DCE022C2A
:102C770084906DDE022C84906DEE022C8405A29068
:102C870000527B10128B392220020122C2059001CB
:102C970078E0F904120CAAF0C202122E50122D6E1F
:102CA7002220030122C205900178E0F914120CAA30
:102CB700F0C203122E50122D6E22E0B48003022CB4
:102CC700DA50FB122CED900050128B7290004F746B
:102CD70050F022C3947F122CED900050128B72900B
:102CE700004F7455F022B420012240FDB43F04C3C5
:102CF70094202240FAC3944075F00884E5F004223A
:102D0700E01475F005A4902D11737410022D43740F
:102D17000C022D437405022D437407022D437409D9
:102D2700022D43740A022D43740B022D43740D02C6
:102D37002D43740E022D43740F022D4390004D1244
:0E2D47008B7222900178122CC19006D0122DB2
:102D550007900178E06004122DE22290684805A2F0
:102D65009000527B10128B3922900178E0B48003D9
:102D7500022D8050FB122DA5022D83128EB99001D4
:102D85008FE0600122900183E0F490019AF09001B8
:102D950082E0F4900199F09006D0E09006D1F022FF
:102DA500900178E0701390019AE0F4900183F0901F
:102DB5000199E0F4900182F022900178122DCE90D5
:102DC5000183F0900182EFF022E075F002A4141463
:102DD500FB9072A093FFEB049072A09322122E8FAA
:102DE500900182122DF5122E96900183122E172234
:102DF5007408C39FFBE005A290005223FAA2E012DB
:102E05002E48F0A3EADFF4EB7001227420F0A3DB77
:102E1500FA22EF700C7B0890005A7420F0A3DBFABD
:102E2500227408C39FFBE005A290005A23FAA2E092
:102E3500122E48F0A3EADFF4EB7001227420F0A310
:102E4500DBFA22400374A52274FF22900178E0701A
:102E5500099006D1E09006D0F022B48006C3947F95
:102E6500022E6A50F8122E729006D0F022B420037A
:102E750074012240FBB43F0374022240FBC394401B
:102E850075F008842403120A92229006D0122E9D12
:102E9500229006D0122EC522E01475F003A4902EC0
:102EA500A7737F08227F08227F05227F07227F08DC
:102EB500227F08227F08227F08227F08227F08229E
:102EC500E01475F003A4902ECF737F08227F0422AF
:102ED5007F00227F00227F01227F02227F03227F43
:102EE50005227F06227F072220020122C2059001CA
:102EF50079E004120CB6F0C202D24A222003012264
:102F0500C205900179E014120CB6F0C203D24A2230
:102F1500900179E014B410057460022F2850F990DF
:102F2500714E93900186F022122F15900179E014CD
:102F350075F006A4902F3D7390703E022FFD9070A2
:102F45004E022FFD90705E022FFD90706E022FFDD8
:102F550090707E022FFD90708E022FFD90709E0264
:102F65002FFD9070AE022FFD9070BE022FFD907068
:102F7500CE022FFD9070DE022FFD9070EE022FFD28
:102F85009070FE022FFD90710E022FFD90711E02B2
:102F95002FFD90712E022FFD90713E022FFD907135
:102FA5004E022FFD90715E022FFD90716E022FFD76
:102FB50090717E022FFD90718E022FFD90719E0201
:102FC5002FFD9071AE022FFD9071BE022FFD907105
:102FD500CE022FFD9071DE022FFD9071EE022FFDC6
:102FE5009071FE022FFD90720E022FFD90721E024F
:102FF5002FFD90722E022FFD05A29000527B10121C
:103005008B392220020122C205900175E004120BC2
:10301500EFF0C202D2322220030122C205900175CF
:10302500E014120BEFF0C203D23222900175E014C6
:1030350060061475F003840475F006A4903045739A
:10304500906DCE02305D906DDE023068906DEE02BF
:103055003068906DFE02306805A29000527B101218
:103065008B392205A29000527B0F128B3990017586
:10307500E014700122123084900061128B6E229050
:103085000175E01470037A0022B4040302309E50E7
:10309500037A0122B407005006C394037A0222C3BF
:1030A50094067A032220020122C205900176E004EB
:1030B500120CC9F0C202D2322220030122C20590AD
:0E30C5000176E014120CC9F0C203D232229040
:1030D30067CF05A29000527B07128B39900176E0EF
:1030E300900059128B6E906E1605A290005A7B08C1
:1030F300128B392220020122C205900177E00412CB
:103103000C15F0C2022220030122C205900177E0D0
:1031130014120C15F0C20322900177E0FA747FC3F6
:103123009AB47F0302313F906E2E05A29000527B2A
:103133000D128B39EA90005F128B8722906DCE05BA
:10314300A29000527B10128B392220020122C20569
:1031530090017AE004120CDCF0C202222003012267
:10316300C20590017AE014120CDCF0C20322900134
:103173007AE0B408041231962240FAB40906907139
:103183006F0231B1B40A0690717F0231B190718F31
:103193000231B190715F05A29000527B0F128B39FF
:1031A30090017AE0900061128B6E1231E12205A248
:1031B3009000527B10128B392290017AE0B40804FC
:1031C3000231E12240FAB409061266A90231E5B4DC
:1031D3000A0612669F0231E51266B30231E59001D9
:1031E3007AE014F9900179E01475F008A42990713C
:1031F300DF93900187F02220020122C20590017B18
:10320300E004120C25F0C2022220030122C2059021
:10321300017BE014120C25F0C2032290017BE01421
:10322300B4100302329E50FB75F006A49032337340
:10323300906F2E023293906F3E023293906F4E0244
:103243003293906F5E023293906F6E023293906F5F
:103253007E023293906F8E023293906F9E0232936E
:10326300906FAE023293906FBE023293906FCE0294
:103273003293906FDE023293906FEE023293906F2F
:10328300FE02329390700E02329390701E023293BC
:1032930005A29000527B10128B3922C3940FFA744B
:1032A30080C39AFA90702E05A29000527B0D128B68
:1032B30039EA90005F128B872220020122C2059017
:1032C300017CE004120C71F0C2022220030122C22D
:1032D3000590017CE014120C71F0C2032290017C72
:1032E300E01475F006A49032ED73906E3E0232F94D
:1032F300906E4E0232F905A29000527B10128B3968
:103303002220020122C20590017DE004120C84F008
:10331300C2022220030122C20590017DE014120C97
:1033230084F0C2032290017DE01475F006A490336B
:103333003573906DCE023347906E5E023347906EC5
:103343006E02334705A29000527B10128B39222064
:10335300020122C20590017EE004120C4BF0C2026E
:10336300C2B62220030122C20590017EE014120C92
:103373004BF0C203C2B62290017EE01475F006A49E
:1033830090338773906EBE023399906ECE02339959
:10339300906EDE02339905A29000527B10128B3996
:1033A3002220020122C20590017FE004120C5EF08C
:1033B300C2022220030122C20590017FE014120CF5
:1033C3005EF0C2032290017FE01475F006A49033EF
:1033D300D573906EEE0233DE906EFE05A29000521E
:1033E3007B10128B3922900166E0B4090122B40AE2
:1033F3000122E56B30E524203C0122D232C23C900D
:103403000166E0B408329006A3124BF4E56C04F0B5
:103413009006AF124BF4E56F04F022D23C1234E075
:1034230012355612343F900202E07003856C6D90A2
:1034330004B7E07003856F6E22302F2290726F0500
:0E344300A29000527B09128B39123465900161
:1034510066E0B40304123B3422B40403123B342269
:103461001234D622E56C12349E05A290005B7B02D9
:10347100128B399067CF05A290005D7B01128B39C9
:10348100E56F12349E05A290005E7B02128B39908B
:1034910067CF05A29000607B02128B392275F00480
:1034A100A49034A6739072782290727A2290727CE2
:1034B1002290727E22907280229072822290728477
:1034C10022907286229072882290728A2290728C47
:1034D1002290728E225350FF4350DE4351D722E592
:1034E1006B20E105740002354D20E20574010235BF
:1034F1004D20E305740202354D20E40574060235C2
:103501004DE56A20E005740302354D20E1057404A0
:1035110002354D20E205740502354D20E30574079F
:1035210002354D20E405740802354D20E505740986
:1035310002354D20E605740A02354D20E705740B6E
:1035410002354D205403E56C22E56F22205403F52A
:103551006C22F56F2275F00AA490355E735350FD0D
:103561004350DC4351D7225350FB4350DA4351D7E8
:10357100225350F74350D64351D7225350EF435073
:10358100CE4351D7225350BF43509E4351D722536C
:10359100507F43505E4351D7225351FE4351D6438E
:1035A10050DE225351FD4351D54350DE225351FB8E
:1035B1004351D34350DE225351EF4351C74350DEB1
:1035C100225351BF4351974350DE2253517F435100
:1035D100574350DE2220020122C205900169E00416
:1035E100120B31F0900168F0C2022220030122C2C5
:1035F10005900169E014120B31F0900168F0C203EB
:1036010022E56B20E50122D2541287EA12372412F7
:1036110036CF3008071235D61235EC22900169E019
:10362100B4010A12372B12374012855722B4020A0D
:1036310012389F1238B312855722B4030A12392265
:1036410012393612855722B4040A12396F123981A0
:1036510012855722B4051F12375C1237751206AC5A
:1036610012098B12093512095C9001727405F090F0
:1036710001637401F022B4060A1238551238691236
:10368100855722B4070A12399A1239AC128557228A
:10369100B4080A123A47123A5912855722B4090A54
:1036A100123A72123A8412855722B40A0A123A9DCA
:1036B100123AAF12855722B40B0A123AC8123ADAFB
:1036C10012855722123AF3123B07128557229001B5
:1036D10069E0B4010412375522B402041238C7223A
:1036E100B4030412394A22B4040412399322B405F2
:1036F1000412378E22B4060412389522B40704123C
:1037010039BE22B40804123A6B22B40904123A9663
:1037110022B40A04123AC122B40B04123AEC221266
:103721003B1B22900169E0022B2E20020122C205DF
:1037310090018BE004120BC9F0C202129E9A222062
:10374100030122C20590018BE014120BC9F0C203E0
:10375100129E9A2290018BE0022BD320020122C2F9
:103761000590018FE0F904120CAAF0C2021238256B
:103771001237B22220030122C20590018FE0F91411
:10378100120CAAF0C2031238251237B22290018F0F
:10379100122CC19006D1122D0790018FE060041206
:1037A10038122290685805A29000527B10128B3972
:1037B1002290018FE0B480030237C450FB1237E935
:0E37C1000237C7128ECC900178E06001229092
:1037CF00019AE0F4900183F0900199E0F490018266
:1037DF00F09006D1E09006D0F02290018FE07013A8
:1037EF00900183E0F490019AF0900182E0F490014F
:1037FF0099F02290018F122DCE90019AF09001999D
:10380F00EFF022123847900199122DF512384E9091
:10381F00019A122E172290018FE070099006D0E0C6
:10382F009006D1F022B48006C3947F02383F50F83F
:10383F00122E729006D1F0229006D1122E9D229058
:10384F0006D1122EC52220020122C205900190E05E
:10385F0004120CB6F0C202D24B2220030122C20581
:10386F00900190E014120CB6F0C203D24B229001DB
:10387F0090E014B41005746002389050F990714EB6
:10388F009390019DF02212387D900190E0022F3429
:10389F0020020122C20590018CE004120BEFF0C24E
:1038AF0002D2322220030122C20590018CE01412B1
:1038BF000BEFF0C203D2322290018CE01460061499
:1038CF0075F003840475F006A49038DC73906DCE08
:1038DF000238F4906DDE0238FF906DEE0238FF90E3
:1038EF006DFE0238FF05A29000527B10128B392219
:1038FF0005A29000527B0F128B3990018CE014704F
:10390F00012212391B900061128B6E2290018CE004
:10391F0002308820020122C20590018DE004120CB2
:10392F00C9F0C202D2322220030122C20590018DBA
:10393F00E014120CC9F0C203D232229067CF05A255
:10394F009000527B07128B3990018DE09000591235
:10395F008B6E906E1605A290005A7B08128B39223F
:10396F0020020122C20590018EE004120C15F0C254
:10397F00022220030122C20590018EE014120C15C1
:10398F00F0C2032290018EE002311F20020122C2F9
:10399F0005900191E004120CDCF0C2022220030119
:1039AF0022C205900191E014120CDCF0C2032290A8
:1039BF000191E0B408041239E32240FAB4090690E9
:1039CF00716F0239FEB40A0690717F0239FE907151
:1039DF008F0239FE90715F05A29000527B0F128B00
:1039EF0039900191E0900061128B6E123A2E2205F0
:1039FF00A29000527B10128B3922900191E0B408F3
:103A0F0004023A2E2240FAB409061266A9023A328B
:103A1F00B40A0612669F023A321266B3023A329025
:103A2F000191E014F9900190E01475F008A4299029
:103A3F0071DF9390019EF02220020122C2059001B6
:103A4F0092E004120C25F0C2022220030122C205CB
:103A5F00900192E014120C25F0C20322900192E023
:103A6F0002322220020122C205900193E004120CBF
:103A7F0071F0C2022220030122C205900193E014CB
:103A8F00120C71F0C20322900193E00232E4200283
:103A9F000122C205900194E004120C84F0C20222AC
:103AAF0020030122C205900194E014120C84F0C28D
:103ABF000322900194E002332C20020122C20590D0
:103ACF000195E004120C4BF0C2022220030122C226
:103ADF0005900195E014120C4BF0C2032290019552
:103AEF00E002337E20020122C205900196E004120B
:103AFF000C5EF0C202C2B52220030122C205900162
:103B0F0096E014120C5EF0C203C2B522900196E04B
:103B1F001475F006A4903B2873906F0E0233DE905D
:103B2F006F1E0233DE9067CF05A290004B7B04120D
:0E3B3F008B3922E56B20E50122123B55123B2B
:103B4D008B123BC112297E2220020122C205305365
:103B5D0010900180E004120D02F0900197F0023BED
:103B6D008620540C900180E004120D02F0023B8679
:103B7D00900197E004120D02F0C202D2362220030A
:103B8D000122C205305310900180E014120D02F095
:103B9D00900197F0023BBC20540C900180E0141270
:103BAD000D02F0023BBC900197E014120D02F0C221
:103BBD0003D23622205413900180123BFF123B3466
:103BCD00900180123D22128E1022900197123BFF20
:103BDD00123B34900197123D22128E2322900180C8
:103BED00123BFF123B34900180123D22128E1002C7
:103BFD003BD7E0B42B06907751023D1150F8147568
:103C0D00F006A4903C14739074B1023D0D9074C1F4
:103C1D00023D0D9074D1023D0D9074E1023D0D9069
:103C2D0074F1023D0D907501023D0D907511023D2F
:103C3D000D907521023D0D907531023D0D90754130
:103C4D00023D0D907551023D0D907561023D0D9037
:103C5D007571023D0D907581023D0D907591023D7E
:103C6D000D9075A1023D0D9075B1023D0D9075C180
:103C7D00023D0D9075D1023D0D9075E1023D0D9007
:103C8D0075F1023D0D907601023D0D907611023DCC
:103C9D000D907621023D0D907631023D0D907641CD
:103CAD00023D0D907651023D0D907661023D0D90D5
:103CBD007671023D0D907681023D0D907691023D1B
:103CCD000D9076A1023D0D9076B1023D0D9076C11D
:103CDD00023D0D9076D1023D0D9076E1023D0D90A5
:103CED0076F1023D0D907701023D0D907711023D69
:103CFD000D907721023D0D907731023D0D9077416A
:103D0D00123F6D2205A29000527B10128B3990004C
:103D1D004F7455F022E0B42B03023D3250FB90005E
:103D2D0050128B7222C3942A900050128B7222E58E
:103D3D006B20E50122123D4F123D85123DBB12292C
:103D4D007E2220020122C205305310900181E00431
:103D5D00120D15F0900198F0023D8020540C900149
:103D6D0081E004120D15F0023D80900198E00412DF
:103D7D000D15F0C202D2372220030122C2053053A5
:103D8D0010900181E014120D15F0900198F0023D94
:103D9D00B620540C900181E014120D15F0023DB6C1
:103DAD00900198E014120D15F0C203D23722205461
:103DBD0013900181123DF9123B34900181123F7E27
:103DCD00128E3622900198123DF9123B34900198D3
:103DDD00123F7E128E4922900181123DF9123B3421
:103DED00900181123F7E128E36023DD1E0B437072D
:103DFD00907D7E123D112250F7B42B03023E0E40F2
:103E0D000BC3942B75F006A4903F1E731475F0062A
:103E1D00A4903E2273907A1E023F69907A2E023F43
:103E2D0069907A3E023F69907A4E023F69907A5EC0
:103E3D00023F69907A6E023F69907A7E023F6990E7
:103E4D007A8E023F69907A9E023F69907AAE023F68
:103E5D0069907ABE023F69907ACE023F69907ADE10
:103E6D00023F69907AEE023F69907AFE023F6990B7
:103E7D007B0E023F69907B1E023F69907B2E023FB5
:103E8D0069907B3E023F69907B4E023F69907B5E5D
:103E9D00023F69907B6E023F69907B7E023F699085
:103EAD007B8E023F69907B9E023F69907BAE023F05
:0E3EBD0069907BBE023F69907BCE023F699008
:103ECB007BDE023F69907BEE023F69907BFE023FF7
:103EDB0069907C0E023F69907C1E023F69907C2E9C
:103EEB00023F69907C3E023F69907C4E023F699095
:103EFB007C5E023F69907C6E023F69907C7E023F44
:103F0B0069907C8E023F69907C9E023F69907CAEEB
:103F1B00023F69907CBE023F69907CCE023F699064
:103F2B007CDE023F69907CEE023F69907CFE023F93
:103F3B0069907D0E023F69907D1E023F69907D2E38
:103F4B00023F69907D3E023F69907D4E023F699032
:103F5B007D5E023F69907D6E023F69907D7E123FD0
:103F6B006D2205A29000527B10128B3990004F747A
:103F7B0050F022E0B43703023F8E50FB90005012FA
:103F8B008B7222C39436900050128B722220020146
:103F9B0022C20590016CE004120B57F0C2022220E2
:103FAB00030122C20590016CE014120B57F0C203FF
:103FBB0022E56B20E501221285571287EA12402178
:103FCB00124004300807123F98123FAA2290016C4E
:103FDB00E0B4010A30500612405412406622B4027B
:103FEB00071240B41240C922B40307124115124103
:103FFB00272212415D12416F2290016CE0B4010443
:10400B0012407822B402041240EB22B40304124192
:10401B0039221241812290016CE01475F006A490B4
:10402B00402E73906ADE024046906AE8024046904A
:10403B006AF2024046906AFC024046122B9B05A294
:10404B009000487B0A128B392220020122C2059074
:10405B000173E004120A4CF0C2022220030122C2B7
:10406B0005900173E014120A4CF0C203229001E791
:10407B00E0B4021A9067CF05A29000527B0D128B11
:10408B0039900173E0241490005F128B87229067A4
:10409B00CF05A29000527B0A128B39906B1A05A2A6
:1040AB0090005C7B06128B392220020122C2059004
:1040BB0001E7E004120C38F0C2021240DE222003AA
:1040CB000122C2059001E7E014120C38F0C2031272
:1040DB0040DE229001E7E0147003C25022D250223E
:1040EB009001E7E01475F006A49040F873906B1AFA
:1040FB0002410A906B2A02410A906B3A02410A056F
:10410B00A29000527B10128B392220020122C20591
:10411B00D25A9001E8E0D2E2F0C20222200301223F
:10412B00C205C25A9001E8E0C2E2F0C203229067D6
:10413B00CF05A29000527B0A128B39205A06906B46
:10414B004A024152906B5005A290005C7B06128B89
:10415B00392220020122C2059001E6E004120B6A0B
:10416B00F0C2022220030122C2059001E6E01412E4
:10417B000B6AF0C203229067CF05A29000527B0A14
:10418B00128B399001E6E01475F006A490419B73F5
:10419B00906B560241AA906B4A0241AA906B500554
:1041AB00A290005C7B06128B392220020122C205F1
:1041BB0090016DE004120BA3F0C202222003012236
:1041CB00C20590016DE014120BA3F0C20322E56B44
:1041DB0020E501221285571287EA12422A12421455
:1041EB003008071241B51241C72290016DE0B401AE
:1041FB000712428412429622B40207124417124449
:10420B0029221245AA1245BC2290016DE0B401048B
:10421B001242A822B4020412443B221245CE229031
:10422B00016DE01475F006A490423773906B5C023D
:0E423B004249906B66024249906B7002424904
:10424900122B9B05A29000487B0A128B3922300859
:104259002205A290016DE0B4010B9001E3E0900604
:10426900CDF0024279B402089001E4E09006CEF064
:1042790005A222200501229067EF2220020122C215
:10428900059001E3E004120BDCF0C20222200301D5
:1042990022C2059001E3E014120BDCF0C203229064
:1042A90001E3E01475F006A49042B573906BBC026B
:1042B9004381906BC7024381906BD2024381906B1B
:1042C900DD024381906BE8024381906BF3024381E5
:1042D900906BFE024381906C09024381906C140239
:1042E9004381906C1F024381906BD202439F906B74
:1042F900DD02439F906BE802439F906BF302439F5B
:10430900906BFE02439F906C0902439F906BD2020F
:1043190043BD906BDD0243BD906BE80243BD906BDA
:10432900F30243BD906BFE0243BD906C090243BD8D
:10433900906BD20243DB906BDD0243DB906BE802AA
:1043490043DB906BF30243DB906BFE0243DB906C23
:10435900090243DB906BD20243F9906BDD0243F90A
:10436900906BE80243F9906BF30243F9906BFE02FC
:1043790043F9906C090243F912425705A29000577C
:104389007B0B128B39906B8A12425705A29000520F
:104399007B05128B392212425705A29000577B0BDD
:1043A900128B39906B8F12425705A29000527B05F0
:1043B900128B392212425705A29000577B0B128BA0
:1043C90039906B9412425705A29000527B05128BCB
:1043D900392212425705A29000577B0B128B399054
:1043E9006B9912425705A29000527B05128B392214
:1043F90012425705A29000577B0B128B39906B9E86
:1044090012425705A29000527B05128B39222002D5
:104419000122C2059001E4E004120BDCF0C2022281
:1044290020030122C2059001E4E014120BDCF0C262
:1044390003229001E4E01475F006A49044487390B7
:104449006BBC024514906BC7024514906BD20245B0
:1044590014906BDD024514906BE8024514906BF3E0
:10446900024514906BFE024514906C0902451490A4
:104479006C14024514906C1F024514906BD20245CE
:1044890032906BDD024532906BE8024532906BF356
:10449900024532906BFE024532906C09024532901A
:1044A9006BD2024550906BDD024550906BE8024596
:1044B90050906BF3024550906BFE024550906C0989
:1044C900024550906BD202456E906BDD02456E90AD
:1044D9006BE802456E906BF302456E906BFE0245E8
:1044E9006E906C0902456E906BD202458C906BDD23
:1044F90002458C906BE802458C906BF302458C90D9
:104509006BFE02458C906C0902458C12425705A23C
:104519009000577B0B128B39906BA312425705A25F
:104529009000527B05128B392212425705A2900046
:10453900577B0B128B39906BA812425705A290003A
:10454900527B05128B392212425705A29000577BE4
:104559000B128B39906BAD12425705A29000527B1A
:1045690005128B392212425705A29000577B0B1274
:104579008B39906BB212425705A29000527B0512FB
:104589008B392212425705A29000577B0B128B39A7
:10459900906BB712425705A29000527B05128B39D6
:1045A9002220020122C205900171E004120BB6F02B
:0E45B900C2022220030122C205900171E0140B
:1045C700120BB6F0C20322906B7A05A29000527BC1
:1045D7000E128B39900171E014900060128B6E906F
:1045E7006B8905A29000617B01128B391245F72276
:1045F700300E0122900171E01475F00CA412060B25
:10460700C2AD858244858345858246858347D2AD81
:10461700900171E01475F00CA4120623C2AD8582D7
:104627004885834985824A85834B85824C85834D9E
:1046370085824E85834FD2AD22900167E0F91246FD
:104647004BE9F022E56B44E1F47006E56AF4701576
:104657002230E10379012230E2012230E3037902BB
:104667002230E40122E56AF430E0012230E10379E7
:10467700032230E20379042230E30379052230E490
:10468700012230E50379062230E60379082230E774
:104697000379072222C0E0858237858338783790EF
:1046A7000167E014F53B753C00793B12038E868267
:1046B700088683D0E022900167E0900047128B6E56
:1046C7009000487420F02220020122C20590016E5A
:1046D700E004120B44F0C2022220030122C205901B
:1046E700016EE014120B44F0C20322E56B20E601D1
:1046F7002220E501221246401246BD1247471247C3
:10470700313008071246CE1246E02290016EE0B41F
:10471700010712478212479E22B402071249561216
:10472700496E221249EB124A002290016EE0B40151
:10473700041247E822B4020412498622124A1522BB
:1047470090016EE01475F006A490475473906A6E5A
:10475700024774906A79024766906A830247661235
:104767002B9B05A29000497B09128B3922122B9BA8
:1047770005A29000487B05128B392220020122C234
:10478700059001A212469CE0F904120CAAF0C2029D
:104797001247BA12481E2220030122C2059001A225
:1047A70012469CE0F914120CAAF0C2031247BA127F
:1047B700481E229001A212469CE0700F9006D2126A
:1047C70048AEE09006D212469CF022B48006C3940D
:1047D7007F0247DD50F8122E729006D212469CF0E7
:1047E700229001A212469C122CC19006D212469C1E
:1047F700122D079001A212469CE06004124929225B
:1048070090686805A29000527B0F128B391248F20C
:10481700900061128B6E229001A212469CE0B48038
:104827000302483350FB12486D024836128EDF9060
:1048370001A21248AEE06001229001D4124904E0BF
:10484700F49001D41248CEF09001D3124904E0F459
:104857009001D31248CEF09006D212469CE0900603
:10486700D21248AEF0229001A212469CE0701F902F
:1048770001D41248CEE0F49001D4124904F090011B
:10488700D31248CEE0F49001D3124904F0229001EC
:10489700A212469C122DCE9001D4124904F0900129
:1048A700D3124904EFF022C0E08582378583387838
:1048B700371248F214F53B753C00793B12038E869C
:1048C70082088683D0E022C0E085823785833878E6
:1048D700371248F21475F002A4F53B753C00793B9A
:1048E70012038E8682088683D0E022900167E0B4A7
:1048F7000506C3940402490350F8240422C0E08546
:1049070082378583387837900167E01475F002A401
:10491700F53B753C00793B12038E8682088683D06F
:10492700E0221249429001D3124904122DF512498F
:0E4937004C9001D4124904122E17229006D281
:1049450012469C122E9D229006D212469C122EC50E
:104955002220020122C2059001AA12469CE00412FF
:104965000CB6F0C2021249B22220030122C2059000
:1049750001AA12469CE014120CB6F0C2031249B209
:10498500221249949001AA12469CE0122F342290DB
:1049950001AA12469CE014B4100574600249AA509D
:1049A500F990714E939001BA12469CF022900167DE
:1049B500E01475F005A49049BF7379010249E479C3
:1049C500020249E479040249E479080249E47910CC
:1049D5000249E479200249E479400249E47980906A
:1049E50001C2E049F02220020122C2059001C31252
:1049F500469CE004120CDCF0C2022220030122C214
:104A0500059001C312469CE014120CDCF0C203228F
:104A15009001C312469CE0B40804124A3D2240FAB4
:104A2500B4090690716F024A5BB40A0690717F0261
:104A35004A5B90718F024A5B90715F05A2900052AC
:104A45007B0F128B399001C312469CE090006112D6
:104A55008B6E124A8E2205A29000527B10128B3962
:104A6500229001C312469CE0B40804024A8E2240FB
:104A7500FAB409061266A9024A95B40A0612669F97
:104A8500024A951266B3024A959001C312469CE00C
:104A950014FF9001AA12469CE01475F008A42F900B
:104AA50071DF939001CB12469CF02220580122C25F
:104AB50058124B064350DE4351D7E550C2E0F5503E
:104AC500D23AD23AD23B124B1B12852712571812F3
:104AD5004B3A12853F125ED6C232124AE32290014A
:104AE50070E0B4010990020F128675028569B4025F
:104AF500099004C412869E0285694350DE4351D74E
:104B0500229006A3124BF4E014F56C9006AF124BFD
:104B1500F4E014F56F2290068B124BF4E0B43A08DA
:104B2500900180F012912D2240F6C3943A900181B4
:104B3500F012955122900697124BF4E0B43A089082
:104B45000197F01291E22240F6C3943A900198F051
:104B550012956922E56B20E50122900170E0B4030E
:104B6500012290016FE0F9124B72E9F022E56B44E6
:104B7500E1F47008E56AF47028C2592220596FD211
:104B85005930E1057901024BF030E2057902024B1B
:104B9500F030E3057903024BF030E4057907024B69
:104BA500F020594AD259E56AF430E0057904024B00
:104BB500F030E1057905024BF030E2057906024B4C
:104BC500F030E3057908024BF030E4057909024B32
:104BD500F030E505790A024BF030E605790B024B1A
:104BE500F030E705790C024BF0790CD2582222C03F
:104BF500E0858237858338783790016FE014F53B7F
:104C0500753C00793B12038E8682088683D0E022AC
:104C150090016FE0900047128B722220020122C2A0
:104C250005900170E004120B90F0C202124AE322D3
:104C350020030122C205900170E014120B90F0C20E
:104C450003124AE322E56B20E50122E56B20E6012C
:104C550022124B59124CB7124C95300807124C20B2
:104C6500124C3522900170E0B4010C124CF2124D39
:104C750009C254124AE322B4020C124D8D124DA4FE
:104C8500D254124AE322124DF8124E0A124AE32276
:104C9500900170E0B4010A124C15124E34124D20E9
:104CA50022B4020A124C15124E5E124DBB22124E50
:0E4CB5001C22900170E01475F006A4904CC40F
:104CC30073906879024CD690687C024CD6906888C1
:104CD300024CE4122B9B05A29000497B01128B39F5
:104CE30022122B9B05A29000467B0C128B392220AB
:104CF300020122C20590068B124BF4E004120D2828
:104D0300F0D258C2022220030122C20590068B1260
:104D13004BF4E014120D28F0D258C20322124D2492
:104D23002290068B124BF4E0B43A13123C00900627
:104D33008B124BF4123D22906880124D5D2240EBA2
:104D4300C3943A123DFA90068B124BF4E0C3943AA3
:104D5300123F7F906882124D5D2205A290004E7B28
:104D630001128B392290687E05A29000487B0212C3
:104D73008B399006BCE090004A128B729067CF0586
:104D8300A290004C7B01128B392220020122C20522
:104D9300900697124BF4E004120D28F0D258C20289
:104DA3002220030122C205900697124BF4E014124D
:104DB3000D28F0D258C20322124DBF22900697123B
:104DC3004BF4E0B43A13123C00900697124BF412E2
:104DD3003D22906880124D5D2240EBC3943A123D10
:104DE300FA900697124BF4E0C3943A123F7F90680F
:104DF30082124D5D2220020122C2059006BBE0040F
:104E0300120D74F0C2022220030122C2059006BBD8
:104E1300E014120D74F0C203229067CF05A2900034
:104E2300527B0E128B399006BBE0900060128B729E
:104E3300229067CF05A290004A7B01128B39E56C63
:104E430012349E05A290004B7B02128B399067CFE0
:104E530005A290004D7B01128B39229067CF05A2EA
:104E630090004A7B01128B39E56F12349E05A290A4
:104E7300004B7B02128B399067CF05A290004D7BCC
:104E830001128B392220020122C205900172E00433
:104E9300120B7DF0C2022220030122C2059001728F
:104EA300E014120B7DF0C20322303C01221285571D
:104EB3001287EA124F37124F0612510D30080712AC
:104EC3004E88124E9A22900172E01475F003A4905A
:104ED3004ED673024EE5024EEA024EF1024EF8023E
:104EE3004EFFC202C20322124FCC124FDE22124FD8
:104EF300FB12500D2212502A125036221250DC128D
:104F030050E822900160E0600122906A2605A29099
:104F130000527B10128B3922906A3605A290005200
:104F23007B10128B39229067BF05A29000527B1031
:104F3300128B3922900172E01475F006A4904F444D
:104F4300739069F4024F629069FE024F70906A0891
:104F5300024F81906A12024F92906A1C024FAF1265
:104F63002B9B05A29000487B0A128B3922122B9BA4
:104F730005A29000487B08128B39124FF022122BA6
:104F83009B05A29000487B08128B3912501F2212F6
:104F93002B9B05A29000487B05128B399006D012FB
:104FA3002D07745590004FF012510222122B9B05CE
:104FB300A29000487B05128B399006D1122D0774FD
:104FC3005590004FF01251022220020122C2059097
:104FD3000161E004120A7FF0C2022220030122C20F
:104FE30005900161E014120A7FF0C203229001616F
:104FF300E0900050128B722220020122C205900120
:1050030062E004120A7FF0C2022220030122C205D9
:10501300900162E014120A7FF0C20322900162E061
:10502300900050128B722220020122C205125042BC
:0E503300C2022220030122C205125049C2030C
:10504100229006D0125050229006D012509622E0A3
:105051001475F003A490505A7302507802508202E2
:10506100508C02508C02508C02508C02508C025099
:105071008C02508C02508C900163E004120AA5F05E
:1050810022900163E004120AB8F022900163E00467
:10509100120ACBF022E01475F003A49050A0730221
:1050A10050BE0250C80250D20250D20250D2025019
:1050B100D20250D20250D20250D20250D290016399
:1050C100E014120AA5F022900163E014120AB8F06C
:1050D10022900163E014120ACBF02220020122C2C5
:1050E100051250F4C2022220030122C2051250FB14
:1050F100C203229006D1125050229006D11250962E
:1051010022900163E0900050128B7222E56B30E532
:10511100089001E8E0C2E0F0229001E8E020E043DD
:10512100D2E0F0124F2912037D900172E0B401091F
:10513100128F28128F1802515BB4020612516502B8
:10514100515BB4030612517002515BB40406125252
:105151008302515B12529702515B124F1B90016007
:105161007404F02220540412517B221251BD2220DA
:1051710054041251FF221252412290065405A2906A
:105181000202E0120A6FFA9001EA05A2F0A370058B
:105191007C010251AC05A2E0C3940CC3956CA3053C
:1051A100A2F0A3DAF0900202E004FC900161128FF8
:1051B100D005A2ECFB900654128DDC22900661050D
:1051C100A29004B7E0120A6FFA90049F05A2F0A31F
:1051D10070057C010251EE05A2E0C3940CC3956FEA
:1051E100A305A2F0A3DAF09004B7E004FC900161FA
:1051F100128FD005A2ECFB900661128DDC22900685
:105201006E05A2900202E0120A6FFA9001EA05A26D
:10521100F0A370057C0102523005A2E0C3940CC3D7
:10522100956CA305A2F0A3DAF0900202E004FC90D1
:10523100016212904105A2ECFB90066E128DDC22F8
:1052410090067B05A29004B7E0120A6FFA90049FC2
:1052510005A2F0A370057C0102527205A2E0C3947D
:105261000CC3956FA305A2F0A3DAF09004B7E00494
:10527100FC90016212904105A2ECFB90067B128D1D
:10528100DC229006D012908F1290C105A27B029071
:105291000182128DDC229006D112908F1290C105ED
:1052A100A27B02900199128DDC221252B8E56B208B
:1052B100E60122124B592290689405A29000427B8C
:1052C10001128B3990016FE0900043128B7290674D
:1052D100CF05A29000457B01128B39E56C12349EFB
:1052E10005A29000467B02128B399067CF05A290F0
:1052F10000487B01128B3912535F9067CF05A29052
:10530100004D7B01128B391254999068A405A2902B
:1053110000527B01128B399006BCE0900053128B36
:10532100729067CF05A29000557B01128B39E56F12
:1053310012349E05A29000567B02128B399067CFE2
:1053410005A29000587B01128B391253989067CFB8
:1053510005A290005D7B01128B391254B822900690
:105361008B124BF4E0B43A131253E790068B124BB5
:10537100F41254339068801253D12240EBC3943A13
:105381001253FA90068B124BF4E0C3943A12544D27
:105391009068821253D122900697124BF4E0B43AEE
:1053A1001312540D900697124BF4125466906880B4
:0E53B1001253DC2240EBC3943A1254209006B3
:1053BF0097124BF4E0C3943A1254809068821253C0
:1053CF00DC2205A29000497B01128B392205A290A5
:1053DF0000597B01128B3922B42B0790004A745568
:1053EF00F02250F790004A7450F022B43507900025
:1053FF004A7455F02250F790004A7450F022B42BA3
:10540F000790005A7455F02250F790005A7450F0DC
:10541F0022B4350790005A7455F02250F790005A75
:10542F007450F022E0B42B0302544350FB90004B16
:10543F00128B7222C3942A90004B128B7222B435B6
:10544F000302545C50FB90004B128B7222C39434B6
:10545F0090004B128B7222E0B42B0302547650FB58
:10546F0090005B128B7222C3942A90005B128B7296
:10547F0022B4350302548F50FB90005B128B7222C3
:10548F00C3943490005B128B72223005041254D7F0
:10549F00229067CF05A290004E7B01128B399006A8
:1054AF00CBE090004F128B87223005041255B822A3
:1054BF009067CF05A290005E7B01128B399006CCCE
:1054CF00E090005F128B87229006CDE01475F006F6
:1054DF00A49054E4739068B40255AD9068B8025527
:1054EF00AD9068BC0255AD9068C00255AD9068C4D0
:1054FF000255AD9068C80255AD9068CC0255AD907D
:10550F0068D00255AD9068D40255AD9068D8025559
:10551F00AD9068DC0255AD9068E00255AD9068E43F
:10552F000255AD9068E80255AD9068EC0255AD900C
:10553F0068F00255AD9068F40255AD9068F80255C9
:10554F00AD9068FC0255AD9069000255AD906904AD
:10555F000255AD9069080255AD90690C0255AD909A
:10556F0069100255AD9069140255AD906918025536
:10557F00AD90691C0255AD9069200255AD9069241C
:10558F000255AD9069280255AD90692C0255AD902A
:10559F0069300255AD9069340255AD90693805A256
:1055AF0090004E7B04128B39229006CEE01475F0DA
:1055BF0006A49055C57390694002568E90694402B7
:1055CF00568E90694802568E90694C02568E90699D
:1055DF005002568E90695402568E90695802568E1C
:1055EF0090695C02568E90696002568E90696402D3
:1055FF00568E90696802568E90696C02568E90692D
:10560F007002568E90697402568E90697802568E8B
:10561F0090697C02568E90698002568E9069840242
:10562F00568E90698802568E90698C02568E9069BC
:10563F009002568E90699402568E90699802568EFB
:10564F0090699C02568E9069A002568E9069A402B2
:10565F00568E9069A802568E9069AC02568E90694C
:10566F00B002568E9069B402568E9069B802568E6B
:10567F009069BC02568E9069C002568E9069C4051F
:10568F00A290005E7B04128B392290029BE0700384
:10569F007B002230560A90015CE060041265AB2259
:1056AF00900174E0B4190612570B0256EB90049D4B
:1056BF00E0F57C90049CE004B57C1590017DE0B48E
:1056CF0002069001377400F090049C74000256E1BA
:1056DF0050E9F090049CE0125924E0FB90049EF0F6
:1056EF0012308490015BF090015CEAF090015FE072
:1056FF00B2E0F01265BC90049EE0FB2290049DE0A6
:10570F00126680125924E0FB2290029BE070012266
:10571F00128845900174E01475F003A490572F730D
:0E572F0002577A02581602586902589802581A
:10573D00EF02593F0259770259BC025A01025A1819
:10574D00025AAC025AED025B2B025B73025BB30291
:10575D005BEC025C06025C20025C3D025CEF025DCC
:10576D0058025DE1025E07025E11025E5312577E22
:10577D00221257851257D22290029BE0120D4EFA3B
:10578D007BFF7C0090029C05A290020F128659E0CF
:10579D00A30B30E7FA05A2EBF0A305A20CDAF0ECAF
:1057AD0090049DF0FF2290049DE090029C8582372D
:1057BD008583387837F53B753C00793B12038E862F
:1057CD008208868322900176E0F57C157C7E01B4FB
:1057DD000101221257E7D57CFA22EE75F00CA4FDDB
:1057ED000E1257B3EFFB7C0005A290029CE0A32D97
:1057FD0005A2F0A305A20CECB4FF0590049DF022C8
:10580D00DBEB90049DE02CF02212577E12582012F3
:10581D0058392290049DE0FB90039C05A2EB1412D5
:10582D005924E005A2F0A305A2DBF22290049DE02D
:10583D00FB90029C05A290039CE0A305A2F0A3059A
:10584D00A2DBF62290049DE0FB90039C05A2900242
:10585D009CE0A305A2F0A305A2DBF62212577E124F
:10586D0058201258732290049DE0FC1414FBEC1286
:10587D00592405A290039D7C00E0A305A2F0A30589
:10588D00A20CDBF590049DE02CF02212577E9004C3
:10589D009DE0B402012240FD1258201258AF12585B
:1058AD00392290049DE0FC1414FBEC1258D405A28F
:1058BD0090029D7C00E0A305A2F0A305A20CDBF5F0
:1058CD0090049DE02CF02290039C858237858338CF
:1058DD007837F53B753C00793B12038E868208863E
:1058ED00832212577E90049DE0B402012240FD12E6
:1058FD0058201259032290049DE0FB12592405A251
:10590D0090039CE0A305A2F0A305A2DBF690049DF5
:10591D00E075F002A4F02290029C858237858338D1
:10592D007837F53B753C00793B12038E86820886ED
:10593D00832212577E90049DE0B402012240FD1295
:10594D0058201259561258392290049DE0FB1258D6
:10595D00D405A290029CE0A305A2F0A305A2DBF65C
:10596D0090049DE075F002A4F02212577E90049DE4
:10597D00E0B402012240FD12598B125839229004D5
:10598D009DE0FB14FC7D0090029C05A290039C05FC
:10599D00A2ED1259240DE005A2F0A305A2EC1259B7
:1059AD00241CE005A2F0A31BEB700122DBE1221207
:1059BD00577E90049DE0B402012240FD1259D01291
:1059CD0058392290049DE0FB14FC7D0090029C054B
:1059DD00A290039C05A2EC1259241CE005A2F0A391
:1059ED0005A2ED1259240DE005A2F0A31BEB7001E9
:1059FD0022DBE12212577E90049DE0B40201224089
:105A0D00FD12598B125A6B1258392212577E90047F
:105A1D009DE0B402012240FD1259D0125A2F1258A6
:105A2D00392290049DE0FEFB14FC7D0090029C0544
:105A3D00A2125AA705A2ED1259240DE005A2F00EEF
:105A4D00A305A2EC1259241CE005A2F00EA31BEB3A
:105A5D007004025A6522DBDC90049DEEF022900466
:105A6D009DE0FEFB14FC7D0090029C05A2125AA73E
:105A7D0005A2EC1259241CE005A2F00EA305A2ED1F
:105A8D001259240DE005A2F00EA31BEB7004025A6F
:105A9D00A122DBDC90049DEEF022EB1258D42212F1
:0E5AAD00577E90049DE0B402012240FD125A83
:105ABB00C01258392290049DE014FB7C007D0190AC
:105ACB00029CE0FF05A290039CEFF00CA305A2ED56
:105ADB001259240DE005A2F00CA3DBED90049DEC14
:105AEB00F02212577E90049DE0B402012240FD1279
:105AFB005B011258392290049DE014FB7C0090024C
:105B0B009CE0FF05A290039CEFF00CA305A2EB1207
:105B1B005924E005A2F00CA3DBEE90049DECF022DF
:105B2B0012577E90049DE0B402012240FD125820D2
:105B3B00125873125B451258392290049DE01414CD
:105B4B00FB7C007D0190029CE0FF05A290039CEF83
:105B5B00F00CA305A2ED1259240DE005A2F00CA345
:105B6B00DBED90049DECF02212577E90049DE0B487
:105B7B0002012240FD125820125873125B45125B32
:105B8B00901258392290049DE075F00284FCFB9032
:105B9B00039C05A2EC1258D4E0FF05A2E0CFF0A3C2
:105BAB0005A2EFF0A3DBF12212577E90049DE0B427
:105BBB0001012240FD125BC71258392290049DE06F
:105BCB00FB90039C05A290029CE0A305A2F0A324EA
:105BDB000CF0A305A2DBF290049DE075F002A4F09B
:105BEB002212577E90049DE0B401012240FD125811
:105BFB0020125839125BC71258392212577E900463
:105C0B009DE0B401012240FD125820125873125B23
:105C1B00C71258392212577E90049DE0B40101221D
:105C2B0040FD125820125873125BC7125B9012582A
:105C3B003922125C6090049DE0B4020A1258511292
:105C4B005CAF1258392240F4125C97125C6A125CFA
:105C5B00AF1258392290029BE0120D3B02578C90E9
:105C6B00049DE0FBFDFF7E007C0090039C05A29051
:105C7B00029CE0A305A2F0A305A20CDBF50EEDFB45
:105C8B00EE125924DFEC90049DECF02290049DE081
:105C9B00FB12592405A290029CE0A305A2F0A305D8
:105CAB00A2DBF622900176E014700122FF7D0090BA
:105CBB00049D125CCA90049DE00D8DF0A4F022E0CF
:105CCB00FCFB0DECFB8DF0A41258D405A290039CA9
:105CDB00ED75F00CA4FEE02EA305A2F0A305A2DB4C
:105CEB00EFDFDF22125C6090049DE0B4020A1258D1
:105CFB0051125D181258392240F41258201258399B
:105D0B00125C97125C6A125D181258392290017658
:105D1B00E014700122FF7D0090049D125D3390040E
:105D2B009DE00D8DF0A4F022E0FCFB0DECFB8DF063
:105D3B00A41258D405A290039CEF75F00CA4FEE0BE
:105D4B002EA305A2F0A305A2DBEFDFDF22125785FE
:105D5B0090049DE0B4020A125851125CAF125839EC
:105D6B002240F4125D78125CAF1258392290049DD8
:105D7B00E0FB7C0090039C05A290029CE0A305A293
:105D8B00F00CA305A2DBF590049DE014FB90029DA3
:105D9B00E0A305A2F00CA305A2DBF590029CE02486
:105DAB000CA305A2F00CA305A290049DE01414FB18
:105DBB0090029EE0A305A2F00CA305A2DBF57B02EB
:105DCB0090029CE0240CA305A2F00CA305A2DBF32C
:105DDB0090049DECF02212578590049DE0B4020ACA
:105DEB00125820125D181258392240F4125D7812A5
:105DFB005839125820125D1812583922125E1B1294
:105E0B005CAF12583922125E1B125CAF125E3A2243
:105E1B00900202E070012290049DF0FB90039C0520
:0E5E2B00A29001EAE0A305A2F0A305A2DBF617
:105E39002290049DE0FB90029C05A2EB141258D419
:105E4900E005A2F0A305A2DBF22212577E229005FB
:105E590050E070037B002230570A90015EE0600435
:105E69001265D92290018BE0B41906125EC9025E4F
:105E7900A9900652E0F57C900651E004B57C159096
:105E89000194E0B4020690013A7400F0900651744E
:105E990000025E9F50E9F0900651E01260BEE0FBFF
:105EA900900653F012391B90015DF090015EEAF003
:105EB90090015FE0B2E1F01265EA900653E0FB223F
:105EC900900652E01266801260BEE0FB22900550F7
:105ED900E07001221288F790018BE01475F003A499
:105EE900905EED73025F38025FCB02601E02604D67
:105EF9000260890260D902611102615602619B0246
:105F090061B20262410262820262C00263080263F4
:105F19002C02636502637F0263990263B6026468B7
:105F29000264AC02653502655B0265650265A7120C
:105F39005F3C22125F43125F9022900550E0120DE0
:105F49004EFA7BFF7C0090055105A29004C412868D
:105F590067E0A30B30E7FA05A2EBF0A305A20CDA80
:105F6900F0EC900652F0FF22900652E09005518520
:105F790082378583387837F53B753C00793B1203C6
:105F89008E86820886832290018DE0F57C157C7EC1
:105F990001B4010122125FA5D57CFA22EE75F00C3D
:105FA900A4FD0E125F71EFFB7C0005A2900551E084
:105FB900A32D05A2F0A305A20CDBF4900652E02C58
:105FC900F022125F3C125FD5125FEE22900652E07A
:105FD900FB90039C05A2EB141260BEE005A2F0A39E
:105FE90005A2DBF222900652E0FB90055105A29032
:105FF900039CE0A305A2F0A305A2DBF622900652BA
:10600900E0FB90039C05A2900551E0A305A2F0A333
:1060190005A2DBF622125F3C125FD512602822909E
:106029000652E0FC1414FBEC1260BE05A290039D1D
:106039007C00E0A305A2F0A305A20CDBF5900652B3
:10604900E02CF022125F3C900652E0B4020122409B
:10605900FD125FD5126064125FEE22900652E0FCD9
:106069001414FBEC1258D405A29005527C00E0A34D
:1060790005A2F0A305A20CDBF5900652E02CF02254
:10608900125F3C900652E0B402012240FD125FD536
:1060990012609D22900652E0FB1260BE05A2900399
:1060A9009CE0A305A2F0A305A2DBF6900652E075D9
:1060B900F002A4F02290055185823785833878371C
:1060C900F53B753C00793B12038E86820886832254
:1060D900125F3C900652E0B402012240FD125FD5E6
:1060E9001260F0125FEE22900652E0FB1258D405BE
:1060F900A2900551E0A305A2F0A305A2DBF6900644
:1061090052E075F002A4F022125F3C900652E0B40E
:1061190002012240FD126125125FEE22900652E033
:10612900FB14FC7D0090055105A290039C05A2ED8E
:106139001260BE0DE005A2F0A305A2EC1260BE1C20
:10614900E005A2F0A31BEB700122DBE122125F3C08
:10615900900652E0B402012240FD12616A125FEE1C
:1061690022900652E0FB14FC7D0090055105A29097
:10617900039C05A2EC1260BE1CE005A2F0A305A2D7
:10618900ED1260BE0DE005A2F0A31BEB700122DB4E
:10619900E122125F3C900652E0B402012240FD1256
:0E61A9006125126205125FEE22125F3C900625
:1061B70052E0B402012240FD12616A1261C9125F06
:1061C700EE22900652E0FEFB14FC7D00900551057F
:1061D700A2125AA705A2ED1260BE0DE005A2F00EAD
:1061E700A305A2EC1260BE1CE005A2F00EA31BEBF8
:1061F70070040261FF22DBDC900652EEF02290066B
:1062070052E0FEFB14FC7D0090055105A2125AA72F
:1062170005A2EC1260BE1CE005A2F00EA305A2EDDC
:106227001260BE0DE005A2F00EA31BEB7004026224
:106237003B22DBDC900652EEF022125F3C900652C6
:10624700E0B402012240FD126255125FEE22900671
:1062570052E014FB7C007D01900551E0FF05A29000
:10626700039CEFF00CA305A2ED1260BE0DE005A2A2
:10627700F00CA3DBED900652ECF022125F3C900687
:1062870052E0B402012240FD126296125FEE2290A4
:106297000652E014FB7C00900551E0FF05A2900335
:1062A7009CEFF00CA305A2EB1260BEE005A2F00C78
:1062B700A3DBEE900652ECF022125F3C900652E010
:1062C700B402012240FD125FD51260281262DA1271
:1062D7005FEE22900652E01414FB7C007D019005CE
:1062E70051E0FF05A290039CEFF00CA305A2ED126D
:1062F70060BE0DE005A2F00CA3DBED900652ECF0BA
:1063070022125F3C900652E0B402012240FD125F68
:10631700D51260281262DA126325125FEE22900608
:1063270052125B9322125F3C900652E0B4010122A5
:1063370040FD126340125FEE22900652E0FB90038D
:106347009C05A2900551E0A305A2F0A3240CF0A39D
:1063570005A2DBF2900652E075F002A4F022125F6C
:106367003C900652E0B401012240FD125FD5125F56
:10637700EE126340125FEE22125F3C900652E0B4C9
:1063870002012240FD125FD5126028126340125F9E
:10639700EE22125F3C900652E0B402012240FD1249
:1063A7005FD5126028126340126325125FEE221236
:1063B70063D9900652E0B4020A12600612642812EA
:1063C7005FEE2240F41264101263E3125CAF125FB7
:1063D700EE22900550E0120D3B025F4A900652E014
:1063E700FBFDFF7E007C0090039C05A2900551E019
:1063F700A305A2F0A305A20CDBF50EEDFBEE1260E0
:10640700BEDFEC900652ECF022900652E0FB1260E1
:10641700BE05A2900551E0A305A2F0A305A2DBF6F5
:106427002290018DE014700122FF7D009006521228
:106437006443900652E00D8DF0A4F022E0FCFB0DC2
:10644700ECFB8DF0A41258D405A290039CED75F0D7
:106457000CA4FEE02EA305A2F0A305A2DBEFDFDF6D
:10646700221263D9900652E0B4020A12600612643F
:1064770091125FEE2240F4125FD5125FEE126410A4
:106487001263E3126491125FEE2290018DE01470A3
:106497000122FF7D00900652125D33900652E00DF7
:1064A7008DF0A4F022125F43900652E0B4020A1264
:1064B7006006126428125FEE2240F41264CC126464
:1064C70028125FEE22900652E0FB7C0090039C05A9
:1064D700A2900551E0A305A2F00CA305A2DBF5905D
:1064E7000652E014FB900552E0A305A2F00CA305A9
:1064F700A2DBF5900551E0240CA305A2F00CA3053F
:10650700A2900652E01414FB900553E0A305A2F0F5
:106517000CA305A2DBF57B02900551E0240CA30533
:0E652700A2F00CA305A2DBF3900652ECF022CA
:10653500125F43900652E0B4020A125FD5126491CD
:10654500125FEE2240F41264CC125FEE125FD51298
:106555006491125FEE2212656F126428125FEE22BB
:1065650012656F12642812658E229004B7E07001DF
:1065750022900652F0FB90039C05A290049FE0A395
:1065850005A2F0A305A2DBF622900652E0FB9005DA
:106595005105A2EB141258D4E005A2F0A305A2DB25
:1065A500F222125F3C2290049EE0FB90015BE01416
:1065B500F0600122C25622BA0103D25622BA02075E
:1065C50020E00122D25622BA030720E003D2562248
:1065D50022C25622900653E0FB90015DE014F06064
:1065E5000122C25722BA0103D25722BA020720E17B
:1065F5000122D25722BA030720E103D2572222C231
:106605005722900072E004B410027400F09000620A
:10661500A98229F582E022900076E0FA900073E0E5
:1066250004B40F0274FFF09066F4932A900076F09C
:10663500900075E004B410027400F0F9900076E063
:10664500FA900062E58229F582EAF022900076E070
:10665500FA900074E004B4110274FFF0906703939C
:106665002A900076F01266352212660754016008FA
:10667500126607541F246022747F22F974FF89F083
:1066850084F5F0126607842212660775F0208422CD
:1066950012660775F0338424012212660775F0200F
:1066A5008424012212660775F03F842401221266B4
:1066B5000775F0338424032212660775F0108422CF
:1066C50012660775F01F842212660775F02084F89C
:1066D50012660775F03F842822126607540175F08B
:1066E5000CA42212660775F0558475F00CA42203DC
:1066F5007F2C0C0105712133E6FF0B576818BD0986
:10670500A60D004B5D263585B196114093C8D3463D
:106715004C414D45204152504547474941544F5200
:10672500204D4F44554C45204555524F205241432D
:106735004B2056455253494F4E202D203230313390
:106745002056455253494F4E20312E303020286374
:1067550029627920616D70657265204620204C2084
:10676500204120204D2020452020415250454747BB
:106775004941544F5220323031332020564552532F
:10678500494F4E20312E30332020202020202863F1
:1067950029323031332020202020496E6974206150
:1067A5006C6C2044617461203F204F4B20202020D9
:1067B500202020202020204E4F2020506C65617322
:1067C5006520776169742021202020202020202049
:1067D50020202020202020202020202020202020B4
:1067E50020202020202020202020202020202020A4
:1067F500202020202020202020206F666641525036
:1068050020202042415353202043484F52442053D7
:1068150043414C45204D494449202053455455504A
:1068250020584F55543A204C495354202053415633
:10683500452020504C41594C495354204441544122
:106845002020206D6972726F7265642053657142F4
:106855006173736D6972726F72656420536571201F
:106865004172706D6972726F726564205365712033
:10687500582D313A41203A4220543A633A733A4C02
:106885004953542020202020204C656E6768744CA5
:1068950031322023432063503031204173657154D8
:0E68A500303020204420735531362034736586
:1068B3007141706F72416E74724173657141436CC3
:1068C3006B4164756F4174726941646F74416761B0
:1068D300745631323756726E643173657131436C5D
:1068E3006B3164756F3174726931646F74316761D0
:1068F300743273657132436C6B3264756F327472C8
:106903006932646F74326761743373657133436CD6
:106913006B3364756F3374726933646F7433676197
:10692300743473657134436C6B3464756F3474728F
:106933006934646F7434676174546D706F42706F3F
:1069430072426E74724273657142436C6B4264753A
:106953006F4274726942646F744267617456313274
:106963003756726E643573657135436C6B35647578
:106973006F3574726935646F743567617436736526
:106983007136436C6B3664756F3674726936646F37
:1069930074366761743773657137436C6B3764752D
:1069A3006F3774726937646F7437676174387365EE
:1069B3007138436C6B3864756F3874726938646FFF
:1069C30074386761743E4120203E4220203E41429C
:1069D30020582D3120582D3220582D3320582D3456
:1069E30020582D3520582D3620582D3720582D3836
:1069F3002020204152502B424153533E43686F7233
:106A0300643A5530313E5363616C653A55303141D8
:106A13003E5345513136553031423E53455131365F
:106A2300553031507265737320204B45594E4F5486
:106A3300452021202053544F52414745204F4B209E
:106A43002120202020202020204D4F44454E4F540C
:106A530045524550454154202020202052414E4765
:106A6300452020202020474C494445205345513A96
:106A730031365030312020202020434C4F434B20CF
:106A8300202020202047415445202056454C4F4389
:106A930049545920534551552D4D4F44454C4F4F63
:106AA300502D524553455420204F55542D474154A2
:106AB30045202020204F55542D4356584F55543AC6
:106AC300312031363A5365715030314241535320AE
:106AD300202031363A536571503031202020202058
:106AE30054454D504F20202020202053594E4352CF
:106AF30045435620434C4F434B53454E4420434C50
:106B03004F434B5245435620535953455853454ED3
:106B13004420535953455865787465726E204D6906
:106B23006469436C6F636B20202020696E74657207
:106B33006E20436C6F636B43686F72642054726999
:106B43006767657220496E6E6F726D616C20206895
:106B5300616C662020206F666620555345522D31A7
:106B630020494E20555345522D3220494E2054552D
:106B73004E452D4D4F44455365742043562D4F5577
:106B830054733A202B31564172703A20582D313AC2
:106B930020582D323A20582D333A20582D343A209C
:106BA300426173733A582D353A20582D363A20589E
:106BB3002D373A20582D383A2020202020202047F6
:106BC3004C494445204E4F5445524550454154206D
:106BD300202053455155454E43452020434C4F43B8
:106BE3004B20414C4C2020434C4F434B2044554FAA
:106BF3002020434C4F434B205452492020434C4FB9
:106C0300434B20444F542020202020202047415430
:106C13004556454C4F20312E2E31323756454C4F79
:0E6C230020416363526E6420202020555345AB
:106C3100522D3120202020555345522D32436C6175
:106C4100737369633A2020202020207570436C61A2
:106C5100737369633A20202020646F776E436C61FF
:106C6100737369633A20207570646F776E436C614A
:106C7100737369633A2020646F776E7570436F7028
:106C8100793A2020202075702B646F776E436F70E6
:106C9100793A20202020646F776E2B757050696ED1
:106CA10067506F6E673A2020202020757050696E02
:106CB10067506F6E673A202020646F776E50696E5F
:106CC10067506F6E673A207570646F776E50696EAA
:106CD10067506F6E673A20646F776E75704669749E
:106CE10020526F6F743A20202020207570466974FD
:106CF10020526F6F743A202020646F776E4669745A
:106D010020526F6F743A207570646F776E466974A4
:106D110020526F6F743A20646F776E757046697494
:106D2100204F637461763A20202020757046697483
:106D3100204F637461763A2020646F776E466974E0
:106D4100204F637461763A7570646F776E4669742B
:106D5100204F637461763A646F776E7570536B6917
:106D6100703A2020202020202020207570536B694C
:106D7100703A20202020202020646F776E496E76A3
:106D8100657273696F6E3A202020207570496E76A6
:106D9100657273696F6E3A2020646F776E4F72640B
:106DA100657265643A20202020202075704F72643E
:106DB100657265643A20202020646F776E20202060
:106DC1002020202020202052616E646F6D20202021
:106DD100202020202020202020206F6666202020D7
:106DE100202020202020656163683A2031416C74A5
:106DF10065726E617465203173743A2031416C742F
:106E010065726E61746520326E643A2031202020F3
:106E11002020202032206F6374617665732020204A
:106E2100206D6178696D616C3A20313238506F7232
:106E310074616D2E54696D653A20313237202020FE
:106E4100207374657020627920737465702020202E
:106E51002020202020636F6D62696E65642061745B
:106E610020617270656767696F20656E6420617467
:106E71002073657175656E636520656E64696E74F6
:106E810065726E436C6F636B2F4D4944495472694F
:106E9100676765722D496E2020312F313654726932
:106EA100676765722D496E205469636B735472690B
:106EB100676765722D496E20537465707320205386
:106EC100657175656E6365284761746529202020A9
:106ED1005265736574207065722042617220204191
:106EE1007270656767696F2052657365744F757459
:106EF1002D333A202056656C6F636974794F757430
:106F01002D333A43686F7264206E6F74654F7574E8
:106F11002D343A202056656C6F636974794F75740E
:106F21002D343A43686F7264206E6F74652020209F
:106F31002020206669727374206E6F746520202092
:106F4100202020206C617374206E6F74654163632F
:106F5100656E743A206561636820326E64416363D3
:106F6100656E743A206561636820337468416363B8
:106F7100656E743A206561636820347468416363A7
:106F8100656E743A20656163682035746841636396
:106F9100656E743A20656163682036746841636385
:0E6FA100656E743A206561636820377468413C
:106FAF006363656E743A2065616368203874684165
:106FBF006363656E743A2065616368203974685243
:106FCF00616E646F6D3A202020312E2E3132375290
:106FDF00616E646F6D3A202036342E2E3132375267
:106FEF00616E646F6D3A202037362E2E3132375254
:106FFF00616E646F6D3A202039352E2E3132375243
:10700F00616E646F6D3A203131322E2E313237522C
:10701F00616E646F6D3A2020666F726D756C6120C2
:10702F00202020202020206669783A203132373105
:10703F00205469636B3A20312F36342074726933D0
:10704F00205469636B733A20202020312F3332365E
:10705F00205469636B733A20202020312F31363151
:10706F00325469636B733A2020202020312F38323D
:10707F00345469636B733A2020202020312F34342D
:10708F00385469636B733A2020202020312F323916
:10709F00365469636B733A2020203120626172325B
:1070AF00205469636B733A312F3332207472693411
:1070BF00205469636B733A312F31362074726938FB
:1070CF00205469636B733A20312F38207472693101
:1070DF00365469636B733A20312F342074726933DD
:1070EF00325469636B733A20312F322074726936D0
:1070FF00345469636B733A20312F312074726939BC
:10710F00205469636B733A312F313620646F7431B9
:10711F00385469636B733A20312F3820646F74339E
:10712F00365469636B733A20312F3420646F743790
:10713F00325469636B733A20312F3220646F7401BC
:10714F0003060C183060020408102040091224486E
:10715F002020202020616461707465643A20203300
:10716F0061646170742E72616E646F6D3A312D358A
:10717F0061646170742E72616E646F6D3A312D3877
:10718F0061646170742E72616E646F6D3A332D3865
:10719F0020206669782072616E646F6D3A203438F2
:1071AF0020202020616363656E7420206C6F6E67F2
:1071BF0020202020616363656E742073686F727482
:1071CF002020202020202020206669783A2039387E
:1071DF000101010101010102010101020203030486
:1071EF000101020303040407010203050708090F45
:1071FF000103070A0D11131E01070D141B21273C54
:10720F00010D1B2835434F780101010102020203D2
:10721F00010101020203030501010203040505092F
:10722F0001020406080A0B120104080C101417249B
:10723F000108101820282F48010203040506070C27
:10724F00010305080A0D0F1801050B10151B1F3040
:10725F00010B15202B353F600110203040505FC0CF
:10726F004B45594E4F54453A202043234320442346
:10727F0044204520462346204723472041234120D1
:10728F0042234330206D616A6F7220372020202007
:10729F00520000FFFF800080808888AAAA08081487
:1072AF001422225555EEEEE38EE388C30CDB6F9963
:1072BF0099BABAAB5ADB6EDB6AADADD6D6AAD5A9F1
:1072CF00A9ABABDADA9249BBBBAA9AAAD7CAE2A991
:1072DF00A9FFF08000AAA0AD60A940AD502950AB26
:1072EF00502A50ABC0A240B2C0BEF09200B6A0A0D0
:1072FF00A0249002A09A0089800920BBE0A990A940
:10730F00E0BAE0EAC09240A280B2C0B6D0FEA0F8C8
:0E731F00008000C000E000F000A800B000D028
:10732D0000FE008000AA00D800E000EC00F400D4BC
:10733D0000FF808000AA80DB00ED00F700B680CA58
:10734D0080FFC08000AA808A80EA80A500B580F504
:10735D0080FFE08000AAA0D280EAC0F540F780E768
:10736D0040FFF88000AAA8DB60E770BDA0F7B0F978
:10737D00F0FFFC8000AAA8DB68FDF8EDD8FAB0D4C8
:10738D009CFFFE8000AAAAE9DCEEECF5DABDDCFA82
:10739D00B2030004070C0400040709040004070BE2
:1073AD00040004060B040004080B04000204070487
:1073BD0000040507040004070E030003060C040077
:1073CD0004070A040004060A030005070C04000262
:1073DD000507040002050A030003070C0400030758
:1073ED0009040003070A040003060A040003080A3F
:1073FD0004000203070400030507030003070E043E
:10740D0000030609040003060A030004080C040027
:10741D0004080A030002070C040005070A0300050F
:10742D000A0C020000000002000100000200020030
:10743D00000200030000020004000002000500002D
:10744D000200060000020007000002000800000212
:10745D000009000002000A000002000B00000200FB
:10746D000C000002000000000200010000020002FA
:10747D0000000200030000020004000002000500ED
:10748D0000020006000002000700000200080000D4
:10749D00020009000002000A000002000B000002B9
:1074AD00000C000020202020202020202020204D16
:1074BD00616A6F722020202020202020204D616ADB
:1074CD006F7220362020202020202020204D616A40
:1074DD006F722037202020202020204D616A6F728E
:1074ED0020376235202020202020204D616A6F72C8
:1074FD00203723352020202020202020202020610F
:10750D006464203220202020202020202020206193
:10751D006464203420202020202020202020206181
:10752D006464203920202020202044696D696E6913
:10753D00736865642020202020202020202020201A
:10754D002020203720202020202020202020202017
:10755D00203762352020202020202020202020735D
:10756D0075732034202020202073757320342073F0
:10757D007573203220202020202050656E74617498
:10758D006F6E696320202020202020202020204D98
:10759D00696E6F722020202020202020204D696EE2
:1075AD006F7220362020202020202020204D696E53
:1075BD006F7220372020202020204D696E6F7220A1
:1075CD00372062352020202020204D696E6F7220DB
:1075DD003720233520202020204D696E6F722061C9
:1075ED006464203220202020204D696E6F7220614E
:1075FD006464203420202020204D696E6F7220613C
:10760D00646420392020202044696D696E69736897
:10761D006564203720202020202068616C6620645E
:10762D00696D2037202020202020204175676D6551
:10763D006E74656420202020202020202020202012
:10764D0037202335202020202020202020202073AB
:10765D0075732032202020202020202020372073F9
:10766D0075732034202020202020202020466F7587
:10767D0072746873202020496E74657276616C2077
:10768D0020302D30202020496E74657276616C207B
:0E769D0020302D31202020496E7465727661F8
:1076AB006C2020302D32202020496E74657276615B
:1076BB006C2020302D33202020496E74657276614A
:1076CB006C2020302D34202020496E746572766139
:1076DB006C2020302D35202020496E746572766128
:1076EB006C2020302D36202020496E746572766117
:1076FB006C2020302D37202020496E746572766106
:10770B006C2020302D38202020496E7465727661F4
:10771B006C2020302D39202020496E7465727661E3
:10772B006C20302D3130202020496E7465727661CB
:10773B006C20302D3131202020496E7465727661BA
:10774B006C20302D31322020202020207573657263
:10775B002063686F726408000305070206080B00BC
:10776B0000000006000407080105000000000000EF
:10777B0005000307080100000000000000060003DD
:10778B00070A0409000000000000060003050A06B2
:10779B0007000000000000070004070B01050800AC
:1077AB00000000000C0003070A010204050608098B
:1077BB000B05000204070900000000000000070091
:1077CB0004070B0105080000000000070004080B6C
:1077DB0001060A0000000000050005070A02000070
:1077EB000000000000070004070A02050800000063
:1077FB000000070004070A03060900000000000749
:10780B000003070B02060800000000000500030739
:10781B00080200000000000000050005060A010038
:10782B000000000000000500050708010000000033
:10783B00000000050005070A010000000000000021
:10784B00050003070A050000000000000005000505
:10785B00070A0200000000000000050004070902EF
:10786B0000000000000000070004060A02050800E3
:10787B0000000000070003060A01040800000000D6
:10788B0000070004070A02060800000000000700BA
:10789B0004070902050B000000000004000407099F
:1078AB000000000000000000040004070B000000B3
:1078BB000000000000040004060A000000000000A5
:1078CB000000070003070A0205080000000000047F
:1078DB00000307090000000000000000040003077C
:1078EB000A0000000000000000070003070B020560
:1078FB00080000000000070004070B020509000048
:10790B00000000070002060A030509000000000042
:10791B00070003070A010508000000000007000428
:10792B00070B0206090000000000070004070A020B
:10793B00050900000000070003070A020508000004
:10794B00000000070003060A010508000000000004
:10795B00070003070901050B0000000000070003E7
:10796B00070B0105080000000000090003070902CE
:10797B000406080B000000080004070A01030609AF
:10798B0000000000070004060A01050900000000C2
:10799B0000070004070A02060900000000000500AA
:1079AB00030708010000000000000005000507099F
:1079BB00020000000000000005000407090200009F
:1079CB00000000000005000305070A00000000008E
:1079DB000000050004060A0200000000000000077A
:1079EB000004080A01050700000000000800030658
:1079FB00090104070A00000000060004080A020639
:107A0B00000000000000070004080B02060A00003B
:0E7A1B000000002020202020202020416C6749
:107A2900657269616E20202020202020202041726B
:107A3900616269616E20202020202042616C696E9C
:107A4900657369616E2020202020426C7565732062
:107A59006D616A6F722020202020426C7565732049
:107A69006D696E6F722020202020202042797A6172
:107A79006E74696E65202020202020204368726F73
:107A89006D617469632020202020202020446961D1
:107A9900746F6E696320446F75626C65204861720A
:107AA9006D6F6E696320202020202020456E696754
:107AB9006D6174696320202020202020204567798A
:107AC900707469616E2020202020202048696E642E
:107AD900757374616E2048756E67617269616E2095
:107AE9006D616A6F722048756E67617269616E2097
:107AF9006D696E6F724A6170616E3A206869726170
:107B0900796F7368694A6170616E3A697761746FF8
:107B1900796F7368694A6170616E3A6B756D6F69E7
:107B2900796F7368694A6170616E3A20202020205C
:107B3900696E73656E4A6170616E3A20202020205B
:107B4900796F73656E4A6170616E3A20207269744B
:107B5900737573656E4A6170616E3A2020202072D8
:107B6900796F73656E2020206D616A6F72204C6F8A
:107B7900637269616E2020207375706572204C6F85
:107B8900637269616E202020204C796469616E20DE
:107B99006D696E6F72202020202020202020202057
:107BA9004D616A6F722020202020202020204D6105
:107BB9006A6F7220362020202020202020204D614D
:107BC9006A6F7220372020202020204D616A6F7251
:107BD900203720623520202020202020202020202E
:107BE9004D696E6F722020202020202020204D69B1
:107BF9006E6F7220362020202020202020204D6901
:107C09006E6F72203720204D696E6F722068617225
:107C19006D6F6E69634D6F64653A2020202020499D
:107C29006F6E69616E4D6F64653A20202020204493
:107C39006F7269616E4D6F64653A202020506872D9
:107C4900796769616E4D6F64653A20202020204C68
:107C5900796469616E4D6F64653A204D69786F6C1E
:107C6900796469616E4D6F64653A20202020416511
:107C79006F6C69616E4D6F64653A202020204C6FEE
:107C8900637269616E4E6561706F6C6974616E20B3
:107C99006D616A6F724E6561706F6C6974616E2097
:107CA9006D696E6F72202020202020204E696E653C
:107CB90020546F6E65202020202020204F6374619E
:107CC900746F6E696320202020202020204F726964
:107CD900656E74616C20202020202020204F76655D
:107CE90072746F6E65202020202020202020202003
:107CF90050656C6F6720202020202050656E7461CC
:107D0900746F6E69636D616A6F722050656E74611C
:107D1900746F6E69636D696E6F722050656E746100
:107D2900746F6E696320202020202050726F6D656A
:107D3900746865757320202020202020202053702E
:107D4900616E697368202020202053796D6D6574F8
:107D5900726963616C2020202020202057686F6C95
:107D690065746F6E656C656164696E6757686F6C81
:107D790065746F6E65202020202020757365722040
:107D89007363616C650300040700000000000000D4
:0E7D99000000030004070000000000000000CE
:107DA70000070004070205090B000000000001019D
:107DB700010101010101010101011E1E1E1E1E1EFE
:107DC7001E1E1E1E1E1E01010101010101010101EE
:107DD70001010101010101010101010101010CFF83
:107DE70000FF01FF02FF03FF04FF05FF06FF07FF78
:107DF70008FF09FF0AFF0BFF0CFF0DFF0EFF0FFF28
:107E070010FF11FF12FF13FF14FF15FF16FF17FFD7
:107E170018FF19FF1AFF1BFF1CFF1DFF1EFF1FC2C4
:107E2700A5C2A4C295C2A3E55020160274FF7F081D
:107E37003392A6D2A3C2A3DFF7B2A50000C2A5E57D
:107E47005120160274FF79083392A6C2A3D2A3D990
:107E5700F7D2A40000C2A422C2A6D2A67908C2A360
:107E6700A2A733D2A3D9F7F56AC2A6D2A67908C2C8
:107E7700A3A28033D2A3D9F7F56B22900166E0B4B1
:107E87000303027E9650FB900168E0B4050122903F
:107E97000166E0B4070122B4080122E56B20E50181
:107EA70022E56B20E60122127ED3127F56127FD97C
:107EB70012805C1280DF1281621281E512826812E1
:107EC70082EB12836E1283F112847422E56B30E128
:107ED7000DC217202314D223127F22D23222C223AB
:107EE700201707D217127EF2D232222053062054CF
:107EF7001A027F02127F02127F122290020F12864D
:107F070075E0B2E7F07F00128891229004C41286D0
:107F17009EE0B2E7F07F0012889C2220530620548F
:107F27001C027F32127F32127F4422203A209002B5
:107F37000F1286757400F07F0012880D22203B0E09
:107F47009004C412869E7400F07F001288BF22E559
:107F57006B30E20DC218202414D224127FA5D2322E
:107F670022C224201807D218127F75D2322220533A
:107F77000620541A027F85127F85127F9522900270
:107F870010128675E0B2E7F07F0112889122900403
:107F9700C512869EE0B2E7F07F0112889C2220532B
:107FA7000620541C027FB5127FB5127FC722203AE4
:107FB700209002101286757400F07F0112880D223E
:107FC700203B0E9004C512869E7400F07F01128834
:107FD700BF22E56B30E30DC219202514D22512808C
:107FE70028D23222C225201907D219127FF8D2329D
:107FF7002220530620541A02800812800812801883
:1080070022900211128675E0B2E7F07F0212889182
:10801700229004C612869EE0B2E7F07F0212889C87
:108027002220530620541C02803812803812804ABE
:1080370022203A209002111286757400F07F0212F6
:10804700880D22203B0E9004C612869E7400F07F96
:10805700021288BF22E56A30E00DC21A202614D228
:10806700261280ABD23222C226201A07D21A1280D9
:108077007BD2322220530620541A02808B12808B27
:1080870012809B22900212128675E0B2E7F07F03FE
:10809700128891229004C712869EE0B2E7F07F0310
:1080A70012889C2220530620541C0280BB1280BBDE
:1080B7001280CD22203A209002121286757400F0A9
:1080C7007F0312880D22203B0E9004C712869E74F0
:1080D70000F07F031288BF22E56A30E10DC21B2042
:1080E7002714D22712812ED23222C227201B07D271
:1080F7001B1280FED2322220530620541A02810E10
:1081070012810E12811E22900213128675E0B2E7C9
:0E811700F07F04128891229004C812869EE028
:10812500B2E7F07F0412889C2220530620541C02DB
:10813500813E12813E12815022203A209002131274
:1081450086757400F07F0412880D22203B0E900482
:10815500C812869E7400F07F041288BF22E56A303B
:10816500E20DC21C202814D2281281B1D23222C2BB
:1081750028201C07D21C128181D2322220530620CE
:10818500541A0281911281911281A1229002141236
:108195008675E0B2E7F07F05128891229004C91236
:1081A500869EE0B2E7F07F0512889C2220530620C8
:1081B500541C0281C11281C11281D322203A209020
:1081C50002141286757400F07F0512880D22203B7B
:1081D5000E9004C912869E7400F07F051288BF2296
:1081E500E56B30E40DC21D202914D229128234D248
:1081F5003222C229201D07D21D128204D23222202A
:10820500530620541A0282141282141282242290D8
:108215000215128675E0B2E7F07F0612889122906A
:1082250004CA12869EE0B2E7F07F0612889C2220DF
:10823500530620541C028244128244128256222084
:108245003A209002151286757400F07F0612880D8B
:1082550022203B0E9004CA12869E7400F07F0612FF
:1082650088BF22E56A30E30DC21E202A14D22A12E5
:1082750082B7D23222C22A201E07D21E128287D28C
:10828500322220530620541A0282971282971282B4
:10829500A722900216128675E0B2E7F07F071288D2
:1082A50091229004CB12869EE0B2E7F07F071288F8
:1082B5009C2220530620541C0282C71282C71282B8
:1082C500D922203A209002161286757400F07F0795
:1082D50012880D22203B0E9004CB12869E7400F06E
:1082E5007F071288BF22E56A30E40DC21F202B14D8
:1082F500D22B12833AD23222C22B201F07D21F1251
:10830500830AD2322220530620541A02831A12837A
:108315001A12832A22900217128675E0B2E7F07FBF
:1083250008128891229004CC12869EE0B2E7F07F75
:108335000812889C2220530620541C02834A12836B
:108345004A12835C22203A20900217128675740027
:10835500F07F0812880D22203B0E9004CC12869ED9
:108365007400F07F081288BF22E56A30E50DC2204F
:10837500202C14D22C1283BDD23222C22C202007ED
:10838500D22012838DD2322220530620541A028322
:108395009D12839D1283AD22900218128675E0B25C
:1083A500E7F07F09128891229004CD12869EE0B2F3
:1083B500E7F07F0912889C2220530620541C028373
:1083C500CD1283CD1283DF22203A20900218128627
:1083D500757400F07F0912880D22203B0E9004CDA4
:1083E50012869E7400F07F091288BF22E56A30E686
:1083F5000DC221202D14D22D128440D23222C22D3D
:10840500202107D221128410D23222205306205473
:108415001A028420128420128430229002191286B6
:1084250075E0B2E7F07F0A128891229004CE128699
:108435009EE0B2E7F07F0A12889C22205306205462
:108445001C02845012845012846222203A20900229
:10845500191286757400F07F0A12880D22203B0ED2
:108465009004CE12869E7400F07F0A1288BF22E522
:108475006A30E70DC222202E14D22E1284C3D232C6
:1084850022C22E202207D222128493D232222053D6
:0E8495000620541A0284A31284A31284B32278
:1084A30090021A128675E0B2E7F07F0B12889122D0
:1084B3009004CF12869EE0B2E7F07F0B12889C22D5
:1084C30020530620541C0284D31284D31284E52241
:1084D300203A2090021A1286757400F07F0B1288DE
:1084E3000D22203B0E9004CF12869E7400F07F0B6A
:1084F3001288BF2230321BB4080A9006A3124BF431
:10850300E56C04F0128557128520125718125ED6B7
:10851300C23222128520125718125ED622128527E4
:1085230012853F2290020F12865979007B3CE0307E
:10853300E70109A3DBF8E990029BF0229004C4123F
:10854300866779007B3CE030E70109A3DBF8E9901B
:108553000550F02220540990020F12867502856996
:108563009004C412869EE020E709E550D2E1F5505D
:1085730002857CE550C2E1F550A3E020E709E55010
:10858300D2E2F550028590E550C2E2F550A3E02017
:10859300E709E550D2E3F5500285A4E550C2E3F5BF
:1085A30050A3E020E709E550D2E4F5500285B8E591
:1085B30050C2E4F550A3E020E709E550D2E6F550B8
:1085C3000285CCE550C2E6F550A3E020E709E5506B
:1085D300D2E7F5500285E0E550C2E7F550A3E0206D
:1085E300E709E551D2E0F5510285F4E551C2E0F522
:1085F30051A3E020E709E551D2E1F551028608E5F0
:1086030051C2E1F551A3E020E709E551D2E2F5516A
:1086130002861CE551C2E2F551A3E020E709E551CA
:10862300D2E4F551028630E551C2E4F551A3E020CE
:10863300E709E551D2E6F551028644E551C2E6F574
:1086430051A3E020E709E551D2E7F551028658E549
:1086530051C2E7F55122C3E582956CF582E5839417
:1086630000F58322C3E582956FF582E5839400F5D7
:10867300832212865905A2900164E075F00CA424AC
:108683000C05A28582378583387837F53B753C0026
:10869300793B12038E86820886832212866705A29F
:1086A300900164E075F00CA4240C05A28582378543
:1086B30083387837F53B753C00793B12038E86820D
:1086C30008868322900166E0B403030286DB50FB35
:1086D300900168E0B405012212871AE56B30E603C6
:1086E300C23822E56A30E40630E616C23822303852
:1086F3000122D238900164E014120B04F012855762
:108703002230380122D238900164E004120B04F0C5
:1087130012871A12855722900164E0B40009E551CB
:10872300D2E3D2E5F55122B40109E551C2E3D2E522
:10873300F55122B40209E551C2E3C2E5F55122E540
:1087430051D2E3C2E5F55122E56B30E603C239228B
:10875300E56B30E403C2392230390122D239205388
:108763000F205406B23A12877E22B23B1287A3220D
:10877300B23A12877EB23B1287A322203A1BE550FE
:10878300D2E0F5504350DE4351D71296BCD2328526
:108793006C6D9002027400F022E550C2E0F55022A5
:1087A300203B1BE550D2E0F5504350DE4351D71236
:1087B30096C8D232856F6E9004B77400F022E550EC
:1087C300C2E0F55022203A07E550D2E0F55022E509
:1087D30050C2E0F55022203B07E550D2E0F550228D
:0987E300E550C2E0F550222054DB
:1087EC00041287C8221287D9221288862FFF900282
:1087FC0002E012886BEFF0900202E004120D87F099
:10880C0022900202E0FC1288862FF57C7B009001FE
:10881C00E9A3E00BB57CFA8C7C05A2EB12886B0506
:10882C00A2EBB57C08E57C14900202F02205A2E0D4
:10883C00A305A2F0A30B02882D900202E0FB90018D
:10884C00EAE0256CC3956DF0A3DBF6856C6D229088
:10885C000202E0FB9001EAE0256CF0A3DBF9229028
:10886C0001EA8582378583387837F53B753C00798A
:10887C003B12038E868208868322900164E075F099
:10888C000CA4240C2220E70412880D221287F52256
:10889C0020E7041288BF221288A7221288862FFF95
:1088AC009004B7E012891DEFF09004B7E004120DAC
:1088BC0087F0229004B7E0FC1288862FF57C7B00B1
:1088CC0090049EA3E00BB57CFA8C7C05A2EB12897C
:1088DC001D05A2EBB57C08E57C149004B7F02205CD
:1088EC00A2E0A305A2F0A30B0288DF9004B7E0FB83
:1088FC0090049FE0256FC3956EF0A3DBF6856F6E39
:10890C00229004B7E0FB90049FE0256FF0A3DBF905
:10891C002290049F8582378583387837F53B753CE8
:10892C0000793B12038E868208868322753D00C235
:10893C0000C283C2819000427439F0A3741DF0A36D
:10894C007450F0A3746CF0A37479F0A3740CF0A3BE
:10895C007401F0A37406F0E53DB408FB753D00D23C
:10896C000022E53DB41023200120D201C28174C045
:10897C00F954F053800F4280D282C282E9C454F081
:10898C0053800F4280D282C28222E53DB42021C2A4
:10899C00817480F954F053800F4280D282C282E9F4
:1089AC00C454F053800F4280D282C282753D0022A3
:1089BC00C201A2009281900042E582253DF582E041
:1089CC00F954F053800F4280D282C282E9C454F031
:1089DC0053800F4280D282C282053D221203722242
:1089EC0012037212037212037212037212037212C6
:1089FC00037212037222C2821289E81289E8C281C0
:108A0C00C283120372D282C287C286D285D28412EA
:108A1C000372C2821289E8C281C283120372D282AB
:108A2C00C287C286D285D284120372C2821289E8AE
:108A3C00C281C283120372D282C287C286D285D20D
:108A4C0084120372C2821289E8C281C28312037239
:108A5C00D282C287C286D285C284120372C28212AB
:108A6C0089E8C281C283120372D282C287C286D2C3
:108A7C0085C284120372C2821289E8C281C2831237
:108A8C000372D282D287C286C285C284120372C29A
:108A9C00821289E8C281C283120372D282C287C257
:108AAC0086C285C284120372C2821289E8C281C254
:108ABC0083120372D282D287D286D285C2841203E9
:108ACC0072C2821289E8C281C283120372D282C23C
:108ADC0087C286C285C284120372C2821289E8C21E
:108AEC0081C283120372D282C287C286C285D284AB
:108AFC00120372C2821289E8C281C283120372D23B
:108B0C0082C287C286C285C284120372C282128953
:108B1C00E8C281C283120372D282C287D286D28506
:108B2C00C284120372C2821289E8D2002205A2E426
:108B3C0093A305A2F0A3DBF505A22290675F05A223
:108B4C009000427B20028B3990677F05A2900042F7
:0E8B5C007B20028B399067CF05A29000427BF0
:108B6A0020028B392430F02275F00A84AFF075F0B8
:108B7A000A84E5F02430F0EF2430A3F02275F00ADD
:108B8A0084AFF075F00A842430F0E5F02430A3F0C5
:108B9A00EF2430A3F022128B87A3742CF0EE24303A
:108BAA00A3F022D281C283120372D282D287D286E2
:108BBA00D285D284120372C2821289E8D281C28318
:108BCA00120372D282D287D286D285D284120372DB
:108BDA00C2821289E822128B611203721203721284
:108BEA000372120372120372120372120372128B4D
:108BFA00477550DB7551FF1203721203727550CF1D
:108C0A007551FF1203721203727550DF7551FE120D
:108C1A0003721203727550DF7551FB12037212034D
:108C2A00727550DF7551BF1203721203727550DFED
:108C3A0075517F1203721203727550DF7551EF126C
:108C4A0003721203727550DF7551FD12037212031B
:108C5A007275505F7551FF12037212037275509F3D
:108C6A007551FF1203721203727550D77551FF12B4
:108C7A0003721203727550DD7551FF1203721203EB
:108C8A00727550DF7551FF128B544352FF120372F3
:108C9A001203721203721203721203721203721215
:108CAA000372120372120372120372120372120314
:108CBA007212037212037212037212037212037295
:108CCA0012037212037212037212037212037212E5
:108CDA0003721203721203721203721203721203E4
:108CEA0072120372120372535200128B61120372D0
:108CFA0012037212037212037222120372120372A5
:108D0A0012037212037212037212037212037212A4
:108D1A0003721203721203721203721203721203A3
:108D2A007212037212037212037212037212037224
:108D3A001203721203721203721203721203721274
:108D4A000372120372120372120372120372120373
:108D5A0072120372120372120372120372120372F4
:108D6A001203721203721203721203721203721244
:108D7A00037222E56B30E00122435020E550C2E243
:108D8A00F550E551C2E0F55190679F05A290004267
:108D9A007B10128B399067AF05A29000527B10129C
:108DAA008B39E56B30E0FBE56B30E20630E4170205
:108DBA008DB19067BF05A29000527B10128B3912B9
:108DCA000372128F5322E56B30E4FB120372120313
:108DDA007222E5D220E0FBE0A305A2C2AF75D2025F
:108DEA00F075D200D2AFA305A2DBE722E5D220E0DC
:108DFA00FBC2AF75D202E075D200D2AFA305A2F0D2
:108E0A00A305A2DBE722900180128FF105A27B0D58
:108E1A0090065405A2128DF622900197128FF10541
:108E2A00A27B0D90066105A2128DF6229001811295
:108E3A00906205A27B0D90066E05A2128DF6229015
:108E4A00019812906205A27B0D90067B05A2128DF5
:108E5A00F62290000005A27B0D90065405A2128D01
:108E6A00F690000005A27B0D90066105A2128DF610
:108E7A009000D005A27B0D90066E05A2128DF69089
:108E8A0000D005A27B0D90067B05A2128DF62290DA
:108E9A00029E05A27B3190068B05A2128DF62290C6
:108EAA0002CF05A27B7790017305A2128DF622905C
:108EBA00017812901E05A27B0290018205A2128DF2
:108ECA00F62290018F12901E05A27B02900199054D
:0E8EDA00A2128DF6229001A212469C12901E4A
:108EE80005A29001D31249047B0205A2128DF62235
:108EF8007B0D90065405A290000005A2128DDC227D
:108F08007B0D90066E05A29000D005A2128DDC2282
:108F18007B3190068B05A290029E05A2128DDC2261
:108F28007B7790017305A29002CF05A2128DDC22F7
:108F3800E5D220E0FBEA930A05A2C2AF75D202F09F
:108F480075D200D2AFA305A2DBE622128F66128F7C
:108F58007A128F8E128FA2129792128F2822900067
:108F68000005A27C10907D8E7B0D7A00128F38DC74
:108F7800F4229000D005A27C10907DA87B0D7A0089
:108F8800128F38DCF42290029E05A27C01907DB5F8
:108F98007B317A00128F38DCF4229001A07B7F7934
:108FA80080128FBDA3DBFA9001A17B7F7900128F1D
:108FB800BDA3DBFA22E5D220E0FBE9C2AF75D202FD
:108FC800F075D200D2AFA322E01475F00DA4900082
:108FD800008582378583387837F53B753C00793BC7
:108FE80012038E868208868322E0B42B03028FFC4C
:108FF80050FB742BC3942B75F00DA4900000858250
:10900800378583387837F53B753C00793B12038EFA
:10901800868208868322E0C3948075F002A49001BA
:10902800A08582378583387837F53B753C00793BD6
:1090380012038E868208868322E01475F00DA490B0
:1090480000D08582378583387837F53B753C0079C1
:109058003B12038E868208868322E0B4370302908F
:109068006D50FB7437C3943775F00DA49000D0850C
:1090780082378583387837F53B753C00793B120396
:109088008E868208868322E01475F004A490909955
:10909800739001A0229001E02290021E2290022EDD
:1090A8002290023E2290024E2290025E2290026E90
:1090B8002290027E2290028E22858237858338781C
:1090C80037900163E01475F002A4F53B753C007914
:1090D8003B12038E868208868322C2A5C2A4C2954B
:1090E800C2A3E5527F083392A6D2A3C2A3DFF7B288
:1090F800950000C2952220360122C2364350DE4335
:1091080051D7E550C2E0F55030530BD23AD23B125A
:10911800912D1291E222205406D23A12912D22D298
:109128003B1291E2221296BC9002027400F0856C08
:109138006D900180E0B42B0302916550FB1475F02B
:1091480005A4FB90739E93FA0BEB9305A21291C1B1
:1091580005A2DAF412918912885BD23222128E109B
:10916800900654E0FA70061296BCD23222A3E005AB
:10917800A21291C105A2DAF51291B112885BD2321E
:1091880022900180E01475F005A4FB9001EA05A285
:1091980090739E93FAFF0BEB93240C05A2F0A305A2
:1091A800A2DAF3EF900202F0229001EA05A29006FB
:1091B8005412926E900202F02290021B858237852B
:1091C80083387837F53B753C00793B12038E8682ED
:1091D80008868374FFF01299F7221296C89004B794
:1091E8007400F0856F6E900197E0B42B0302921A19
:1091F80050FB1475F005A4FB90739E93FA0BEB9348
:1092080005A212927F05A2DAF412923612890DD2C3
:109218003222128E23900661E0FAA3E005A2129290
:109228007F05A2DAF512925E12890DD232229001E0
:1092380097E01475F005A4FB90049F05A290739E17
:1092480093FAFF0BEB93240C05A2F0A305A2DAF323
:0E925800EF9004B7F02290049F05A2900661EB
:1092660012926E9004B7F022E0FAFFA3E0240C05F8
:10927600A2F0A305A2DAF4EF229004D08582378506
:1092860083387837F53B753C00793B12038E86822E
:1092960008868374FFF01299F72290029BE0700112
:1092A60022B404030292B140FB74041475F003A4C3
:1092B6009092BA730292C60292E702931602933B09
:1092C6009006BCE0FD9001EAE02D9006BDF0240C6E
:1092D6009006BEF0240C9006BFF0240C9006C0F059
:1092E600227A029006BCE0FD9006BD05A29001EA36
:1092F600E02DA305A2F0A305A2DAF59006BDE024B1
:109306000C9006BFF09006BEE0240C9006C0F0223A
:109316007A039006BCE0FD9006BD05A29001EAE046
:109326002DA305A2F0A305A2DAF59006BDE0240C54
:109336009006C0F0227A049006BCE0FD9006BD05BA
:10934600A29001EAE02DA305A2F0A305A2DAF52278
:109356009006BDE01206238582488583499006BEA5
:10936600E012062385824A85834B90017FE0B40292
:109376000D9006BFE012062385824C85834D900131
:1093860096E0B4020D9006C0E012062385824E8553
:10939600834F2290029BE0B400041293E122B401B1
:1093A6000D1293EE1294651294B21294FF22B40237
:1093B6000D1293EE12943B1294B21294FF22B40350
:1093C6000D1293EE12943B1294881294FF2212937C
:1093D600EE12943B1294881294D522129418129489
:1093E600651294B21294FF221294189006BDE0FF03
:1093F6007492120E0F9006BCE02F2424C2E790064A
:10940600C1F0120E0F7464120E0F9006C5E0D2E082
:10941600F0229006C5E020E001229006C1E0FF742C
:1094260092120E0FEF120E0F7400120E0F9006C559
:10943600E0C2E0F0221294659006BEE0FF7492123C
:109446000E0F9006BCE02F2424C2E79006C2F0124D
:109456000E0F7464120E0F9006C5E0D2E1F0229052
:1094660006C5E020E101229006C2E0FF7492120ECA
:109476000FEF120E0F7400120E0F9006C5E0C2E138
:10948600F0221294B29006BFE0FF7492120E0F9073
:1094960006BCE02F2424C2E79006C3F0120E0F7418
:1094A60064120E0F9006C5E0D2E2F0229006C5E0E7
:1094B60020E201229006C3E0FF7492120E0FEF1213
:1094C6000E0F7400120E0F9006C5E0C2E2F02212D3
:1094D60094FF9006C0E0FF7492120E0F9006BCE057
:1094E6002F2424C2E79006C4F0120E0F7464120EE5
:1094F6000F9006C5E0D2E3F0229006C5E020E30116
:10950600229006C4E0FF7492120E0FEF120E0F7433
:1095160000120E0F9006C5E0C2E3F02220370122AA
:10952600C2374350DE4351D7E550C2E0F5503053C1
:109536000BD23AD23B12955112956922205406D28B
:109546003A12955122D23B129569221296BC90028C
:10955600027400F0856C6D12958112959212885BEB
:10956600D232221296C89004B77400F0856F6E123C
:10957600960712961812890DD23222900181E0B414
:1095860037041295B92250FA1295A922900181E06A
:10959600B437071295B91295E82250F712968D1234
:1095A60095CE2212968D0BEB9305A21291C105A2C0
:1095B600DAF422128E3690066EE0FAFFA3E005A2D8
:1095C6001291C105A2DAF52205A29001EA05A20BC5
:0E95D600EB93240C05A2F0A305A2DAF3EF90AC
:1095E4000202F02290066EE0FFFA05A29001EA055D
:1095F400A2A3E0240C05A2F0A305A2DAF4EF9002E2
:1096040002F022900198E0B4370412963F2250FAF7
:1096140012962F22900198E0B4370712963F1296C3
:109624006E2250F712968D1296542212968D0BEBE1
:109634009305A212927F05A2DAF422128E499006B3
:109644007BE0FAFFA3E005A212927F05A2DAF522DD
:1096540005A290049F05A20BEB93240C05A2F0A392
:1096640005A2DAF3EF9004B7F02290067BE0FFFA4C
:1096740005A290049F05A2A3E0240C05A2F0A30573
:10968400A2DAF4EF9004B7F022B4130302969550D3
:10969400069077610296B2B426030296A35009900D
:1096A4007858C394130296B290794EC394261475D5
:1096B400F00DA4FB93FAFF2274007998900203F052
:1096C400A3D9FC22740079989004B8F0A3D9FC22A1
:1096D4007908F0A3D9FC2274019001A21296D474E3
:1096E400039001AA1296D474069001B21296D4740F
:1096F400069001BA1296D474049001C31296D474DD
:10970400039001CB1296D422740090014B1296D48C
:1097140022740090013B1296D422740090014312EB
:1097240096D422791190007A7400F0A37400F0A307
:10973400D9F6799990009C7400F0A3D9FC22790A97
:109744009006D07401F0A3D9FC22900654029757D6
:1097540090066174057900F07B0CA3E9F009DBFA4B
:109764002290066E02976E90067B74057900F07B5A
:109774000CA3E9F009DBFA90068B12978922900674
:1097840097129789227B0C7401F0A3DBFC22746E80
:10979400900173F07401900174F09001E9F090016C
:1097A40075F0900184F0741190017BF074019001C4
:1097B4008AF090017EF0740290017FF074019001B0
:1097C4007CF090017DF07403900179F074069001AF
:1097D40085F0900186F0740490017AF0740390018E
:1097E40087F07401900176F07402900178F07400AF
:1097F400900177F07400900188F004F074019001F6
:1098040080F07401900181F0740190018BF090015B
:109814008CF090019BF07411900192F0740190010E
:10982400A1F0900195F07402900196F074019001FA
:1098340093F0900194F07403900190F074069001F9
:109844009CF090019DF07404900191F074039001D8
:109854009EF0740190018DF0740290018FF07400F9
:1098640090018EF0740090019FF004F07401900157
:1098740097F0900198F074029001E3F09001E4F005
:1098840012974E12975412976512976B9001E574D4
:1098940000F09001E67402F0C25AD25074029001B2
:1098A400E7F074029001E8F02290017BE014B41018
:1098B40009C3940F7980C9C3992250F575F003A4A4
:1098C4009098C87302994302994302998802998D2A
:1098D40002999202999702999C0299A10299A6026F
:1098E40099AB02994302994B02995302995D0299EB
:1098F40065129971900192E014B41009C3940F7920
:1099040080C9C3992250F575F003A490991373028A
:1099140099430299430299B00299B50299BA0299FE
:10992400BF0299C40299C90299CE0299D3029943FC
:1099340002994B02995302995D0299651299711229
:109944006607547FD2E022126607543F2440221255
:0E995400660775F00584244C22126607541F26
:10996200246022126607541F75F0028424702212AA
:10997200660754016008126607541F2454221266B7
:1099820007540F24702274020299D874030299D8E2
:1099920074040299D874050299D874060299D8748D
:1099A200070299D874080299D874090299D87402E6
:1099B2000299DF74030299DF74040299DF740502CD
:1099C20099DF74060299DF74070299DF740802991D
:1099D200DF74090299DF900188F00299E390019FF8
:1099E200F0F57CA3E004B57C067400F0747F22508D
:1099F200F8F074642222F9900041E0B40001229050
:109A0200003FE0900000F582E9F090003FE004B4EE
:109A12003F027400F0900041E014F022C2AC9000CA
:109A220041E0B43E03D2AC2204F0900040E090004A
:109A320000F582E0F9900040E004B43F027400F0C7
:109A4200D2ACE9120E49029A1E304FD0C24F229078
:109A5200068AE020E00122C2E0F0129A66129A958C
:109A6200129ABC229001E5E030E00122C2AD12045C
:109A7200D8D2AD12047C75F00A8404120BC9F57CAD
:109A82009006C7E0B57C0122E57CF0900174F012EB
:109A9200851622C2AD1204CCD2AD12047C75F03F01
:109AA2008404120CC9F57C9006C8E0B57C0122E55D
:109AB2007CF0900176F0128516229006CDE01475A6
:109AC200F003A4909AC973029B3D029B72029B927F
:109AD200029BAD029BCF029BDC029BE9029BF6023A
:109AE2009C13029C3A029C46029C64029C89029C42
:109AF20096029CA3029CB0029CCD029CEB029D109C
:109B0200029D1D029D2A029D37029D54029D7202F2
:109B12009D97029DA4029DB1029DBE029DDB029D06
:109B2200F9029E1E029E2B029E38029E45029B59FE
:109B3200C2AD1204C0D2AD12047C22129B3275F067
:109B42000284120C15F57C9006CBE0B57C0122E56F
:109B52007CF0900177F022129B32120A5C14F57CA1
:109B62009006CBE0B57C0122E57CF0900173F022F7
:109B7200129B3275F01C8404120BEFF57C9006CB1D
:109B8200E0B57C0122E57CF0900175F01285162289
:109B9200129B32F57C9006CBE0B57C0122E57CF08D
:109BA200900178F0122E50122D6E22129B3275F017
:109BB2000F8404120CB6F57C9006CBE0B57C012232
:109BC200E57CF0900179F0122F15D24A22129B32D5
:109BD20075F03384042401029BB8129B3275F03372
:109BE20084042407029BB8129B3275F0408404243B
:109BF2000D029BB8129B3275F0188404120CDCF52E
:109C02007C9006CBE0B57C0122E57CF090017AF0F5
:109C120022129B3275F0028404120AF1797FC9C3C1
:109C2200992411120C25F57C9006CBE0B57C01221B
:109C3200E57CF090017BF022129B3275F0128424B5
:109C420003029C28129B32F57C9006CBE0B57C0186
:109C520022E57CF09001A2F09001677401F01248B5
:109C62001E22129B3275F00F8404120CB6F57C9002
:109C720006CBE0B57C0122E57CF09001AAF07901E7
:109C82009001C2E049F022129B3275F03384042421
:109C920001029C6F129B3275F03384042407029CEC
:109CA2006F129B3275F0408404240D029C6F129B4C
:109CB2003275F0188404120CDCF57C9006CBE0B50A
:109CC2007C0122E57CF09001C3F022129B32F57CEC
:0E9CD2009006CBE0B57C0122E57CF09001A36A
:109CE000F09001677402F012481E22129B3275F048
:109CF0000F8404120CB6F57C9006CBE0B57C0122F3
:109D0000E57CF09001ABF079029001C2E049F022CD
:109D1000129B3275F03384042401029CF6129B32AC
:109D200075F03384042407029CF6129B3275F040D0
:109D30008404240D029CF6129B3275F01884F57C85
:109D40009006CBE0B57C0122E57C04120CDCF0909F
:109D500001C4F022129B32F57C9006CBE0B57C0169
:109D600022E57CF09001A4F09001677403F01248A2
:109D70001E22129B3275F00F8404120CB6F57C90F3
:109D800006CBE0B57C0122E57CF09001ACF07904D3
:109D90009001C2E049F022129B3275F03384042412
:109DA00001029D7D129B3275F03384042407029DCD
:109DB0007D129B3275F0408404240D029D7D129B20
:109DC0003275F0188404120CDCF57C9006CBE0B5FB
:109DD0007C0122E57CF09001C5F022129B32F57CDB
:109DE0009006CBE0B57C0122E57CF09001A5F090D7
:109DF00001677404F012481E22129B3275F00F8422
:109E000004120CB6F57C9006CBE0B57C0122E57C13
:109E1000F09001ADF079089001C2E049F022129B68
:109E20003275F03384042401029E04129B3275F0D3
:109E30003384042407029E04129B3275F04084048C
:109E4000240D029E04129B3275F0188404120CDC5F
:109E5000F57C9006CBE0B57C0122E57CF09001C654
:109E6000F02290068AE020E30122C2E3F0129E77FE
:109E7000129EA9129ED022C2AD1204F0D2AD1204DD
:109E80007C75F00A8404120BC9F57C9006C9E0B514
:109E90007C0122E57CF090018BF09001E5E030E060
:109EA0000412A31E2212851622C2AD1204B4D2AD32
:109EB00012047C75F03F84F57C9006CAE0B57C0105
:109EC00022E57C04120CC9F090018DF01285162257
:109ED0009006CEE01475F003A4909EDD73029F4EB1
:109EE000029F6A029F8A029FA5029FC7029FD40217
:109EF0009FE1029FEE02A00B02A03202A03E02A050
:109F00005C02A08102A08E02A09B02A0A802A0C5B4
:109F100002A0E302A10802A11502A12202A12F02C0
:109F2000A14C02A16A02A18F02A19C02A1A902A1D7
:109F3000B602A1D302A1F102A21602A22302A2300C
:109F400002A23DC2AD1204E4D2AD12047C22129FE3
:109F50004375F00284120C15F57C9006CCE0B57CBC
:109F60000122E57CF090018EF022129F4375F01CD7
:109F70008404120BEFF57C9006CCE0B57C0122E561
:109F80007CF090018CF012851622129F43F57C9094
:109F900006CCE0B57C0122E57CF090018FF0123810
:109FA000251237B222129F4375F00F8404120CB6AB
:109FB000F57C9006CCE0B57C0122E57CF090019028
:109FC000F012387DD24B22129F4375F03384042463
:109FD00001029FB0129F4375F03384042407029F4F
:109FE000B0129F4375F0408404240D029FB0129F6D
:109FF0004375F0188404120CDCF57C9006CCE0B5B7
:10A000007C0122E57CF0900191F022129F4375F0D3
:10A01000028404120AF1797FC9C3992411120C2514
:10A02000F57C9006CCE0B57C0122E57CF0900192B5
:10A03000F022129F4375F01284240302A020129F85
:10A0400043F57C9006CCE0B57C0122E57CF09001E4
:0EA05000A6F09001677405F012481E22129FC0
:10A05E004375F00F8404120CB6F57C9006CCE0B577
:10A06E007C0122E57CF09001AEF079109001C2E007
:10A07E0049F022129F4375F0338404240102A06735
:10A08E00129F4375F0338404240702A067129F4386
:10A09E0075F0408404240D02A067129F4375F018DA
:10A0AE008404120CDCF57C9006CCE0B57C0122E534
:10A0BE007CF09001C7F022129F43F57C9006CCE015
:10A0CE00B57C0122E57CF09001A7F0900167740643
:10A0DE00F012481E22129F4375F00F8404120CB624
:10A0EE00F57C9006CCE0B57C0122E57CF09001AFCA
:10A0FE00F079209001C2E049F022129F4375F033AF
:10A10E008404240102A0EE129F4375F033840424CC
:10A11E000702A0EE129F4375F0408404240D02A0A6
:10A12E00EE129F4375F0188404120CDCF57C900639
:10A13E00CCE0B57C0122E57CF09001C8F022129FA4
:10A14E0043F57C9006CCE0B57C0122E57CF09001D5
:10A15E00A8F09001677407F012481E22129F4375F3
:10A16E00F00F8404120CB6F57C9006CCE0B57C01A1
:10A17E0022E57CF09001B0F079409001C2E049F008
:10A18E0022129F4375F0338404240102A175129F9D
:10A19E004375F0338404240702A175129F4375F0B2
:10A1AE00408404240D02A175129F4375F018840497
:10A1BE00120CDCF57C9006CCE0B57C0122E57CF03F
:10A1CE009001C9F022129F43F57C9006CCE0B57C3D
:10A1DE000122E57CF09001A9F09001677408F0125D
:10A1EE00481E22129F4375F00F8404120CB6F57CA4
:10A1FE009006CCE0B57C0122E57CF09001B1F079BF
:10A20E00809001C2E049F022129F4375F03384041E
:10A21E00240102A1FC129F4375F03384042407022B
:10A22E00A1FC129F4375F0408404240D02A1FC1280
:10A23E009F4375F0188404120CDCF57C9006CCE07C
:10A24E00B57C0122E57CF09001CAF02290068AE0EE
:10A25E0020E40122C2E4F0D25F12A27412A2901284
:10A26E0092A012939922C2AD120508D2AD12047CAF
:10A27E0075F01584F57C9006BCE0B57C0122E57C7A
:10A28E00F022C2AD1204FCD2AD12047C75F017841C
:10A29E0004F57C9006C6E0B57C0122E57CF0F57CE9
:10A2AE009006BBE0B57C0990016FE57CF0D2582298
:10A2BE0050F52290068AE020E20122C2E2F09001DF
:10A2CE00E5E0B2E0F020E00412A33A2212A3162237
:10A2DE009001E5E020E00412A33A2212A2ED22C280
:10A2EE009190018BE0B4190302A30120E004140243
:10A2FE00A30104900174F0128516229001E5E0206E
:10A30E00E003D29122C29122900174E09001E9F013
:10A31E00C29190018BE0B4190302A33220E0041421
:10A32E0002A33204900174F012851622D29190018C
:10A33E00E9E0900174F01285162243B71843B81263
:10A34E00758790758922758DF8758BF8D28E7598F4
:10A35E0050C299C298D2ACC2117553287554047567
:10A36E00557D75560290FF9C8582CA8583CB85826A
:10A37E00CC8583CD43C804D2ADD2AF2243B7404380
:10A38E00B8408541EA8542FA43D90143DA49755707
:10A39E000875580CD2DED2AE22439C00439D1D435D
:10A3AE00B10122C0E0C0D0E582C0E0E583C0E090FC
:10A3BE00068AE59EF0539EE2D0E0F583D0E0F5826A
:0EA3CE00D0D0D0E032C0E0C0D030DF07C2DF18
:10A3DC00D0D0D0E032C2D8E5EA2541F5EAE5FA352D
:10A3EC0042F5FAD5570B755708D209D5580375584D
:10A3FC000CD0D0D0E032C0E0C0D0E582C0E0E58324
:10A40C00C0E0C2D4D2D3309911C211C299D0E0F5B8
:10A41C0083D0E0F582D0D0D0E032309807C298E5F6
:10A42C00991299F8D0E0F583D0E0F582D0D0D0E045
:10A43C0032C0E0C0D0E582C0E0E583C0E0D2D4C237
:10A44C00D3C2CF201212D55D0F755DFFD55E098585
:10A45C005B5D855C5E122008201312D5630F75635B
:10A46C00FFD564098561638562641222E0D5533B94
:10A47C0075532812051412896E12065312066412B3
:10A48C0090E2D55426755406127E5FB216127E26C3
:10A49C00D55518755532C205900160E0600214F074
:10A4AC00D55608755603D205126651D0E0F583D007
:08A4BC00E0F582D0D0D0E032BF
:00000001FF
